:100000000C9467020C9484020C9484020C94840275
:100010000C9484020C9484020C9484020C94840248
:100020000C9484020C94950D0C9484020C94760D1F
:100030000C9407190C9484020C9484020C9484028E
:100040000C9484020C9484020C948B0C0C94840207
:100050000C9455050C9484020C941F050C94840296
:100060000C94F60E0C9484020C940A180C948402DE
:1000700027182C185D186A186F18711859187A18F3
:10008000A4188B188F18AF189918A41892189618DE
:10009000AF189918A418A818AC18AF18B3180A0A02
:1000A0000D004E65757472616C0048656164696E1F
:1000B00067486F6C64000A0D537465756572756EE0
:1000C000673A20004F4B0A0D000A0D4162676C65CC
:1000D000696368204C756674647275636B73656ED2
:1000E000736F722E2E000A0D42656E75747A65204C
:1000F000506172616D657465727361747A202564F4
:10010000000A0D414343206E696368742061626791
:1001100065676C696368656E21000A0D496E6974D4
:100120002E20454550524F4D3A2047656E65726905
:100130006572652044656661756C742D50617261ED
:100140006D657465722E2E2E000A0D3D3D3D3D3DC0
:100150003D3D3D3D3D3D3D3D3D3D3D3D3D3D3D3DCF
:100160003D3D3D3D3D3D3D3D3D000A0D466C6967D1
:100170006874436F6E74726F6C0A0D4861726477B5
:100180006172653A25642E25640A0D536F66747793
:100190006172653A5625642E2564256320002E0081
:1001A00048693A253469202043663A25346920009D
:1001B00047733A253469202047693A25346920007D
:1001C0004E693A2534692020526F3A25346920005F
:1001D00045787465726E436F6E74726F6C20200088
:1001E00052616E67653A2533692D25336900537472
:1001F000656C6C756E673A202533690053657470C1
:100200006F696E74202025336900536572766F2004
:100210002000506F7469343A202025336900506FF4
:100220007469333A202025336900506F7469323A7B
:10023000202025336900506F7469313A202025331E
:10024000690053746172743A20202020202535699A
:10025000004D657373776572743A20202535690007
:100260005269636874756E673A2020253569004BC2
:100270006F6D706173732020202020202000456D59
:1002800070662E506567656C3A253569005370615C
:100290006E6E756E673A202025356900486F636879
:1002A0002025346920282533692900526F6C6C2081
:1002B000253469202825336929004E69636B202580
:1002C000346920282533692900414343202D2053D8
:1002D000656E736F72004769657220253469202846
:1002E00025336929282533692900526F6C6C202534
:1002F00034692028253369292825336929004E6966
:10030000636B202534692028253369292825336922
:100310002900476965722025346920282533692919
:1003200000526F6C6C202534692028253369290020
:100330004E69636B202534692028253369290047DD
:100340006965722025346920282533692900526F98
:100350006C6C20253469202825336929004E696397
:100360006B20253469202825336929004779726F6D
:10037000202D2053656E736F720050333A25346917
:10038000202050343A253469200050313A25346910
:10039000202050323A253469200047733A253469C9
:1003A000202047693A25346920004E693A2534698E
:1003B0002020526F3A25346920004B373A253469A2
:1003C00020204B383A25346920004B353A253469D2
:1003D00020204B363A25346920004B333A253469C6
:1003E00020204B343A25346920004B313A253469BA
:1003F00020204B323A25346920004B6F6D706173B9
:10040000733A20202025356900526F6C6C3A202009
:1004100020202020253569004E69636B3A2020207A
:1004200020202025356900616B742E204C616765A2
:100430000048F668656E726567656C756E67004B9F
:1004400065696E6520004F66662020202020203AD6
:1004500020253569004C756674647275636B3A20AB
:1004600025356900536F6C6C486F6568653A2025C7
:10047000356900486F6568653A20202020202535C1
:10048000690028632920486F6C6765722042757384
:10049000730053657474696E673A202564200048C0
:1004A000573A5625642E25642053573A25642E2545
:1004B000642563002B204D696B726F4B6F70746500
:1004C00072202B005B25695D005B25695D001124AE
:1004D0001FBECFEFD0E1DEBFCDBF14E0A0E0B1E0A2
:1004E000E6E9FBE802C005900D92A43BB107D9F7FD
:1004F00019E0A4EBB4E001C01D92A237B107E1F707
:100500000E94F6020C94CA450C94000022E030E0F0
:10051000D9010E94B645802D863028F082E0D901AD
:10052000082E0E94BE4590E0089580917B08E82F38
:10053000F0E0EE0FFF1FE35BF74F808191818D5E4E
:100540009F4F14F010920201808191818A5B9F4F2E
:10055000BCF480910201882399F481E08093020128
:10056000809146078F5F80934607853038F088EE8C
:1005700093E09093D6048093D50402C00E94A426F1
:100580008091460790E09093140880931308089593
:10059000FB01282F863008F025E0429FD00111246E
:1005A000AC59BF4F842F90E0019724F001900E9436
:1005B000BE45FACFA2E0B0E0022E0E94BE450E94E6
:1005C000A8400895FB01863008F085E0489FD001DF
:1005D0001124AC59BF4F842F90E0019724F00E9462
:1005E000B6450192FACF0E94A8400895EF92FF927B
:1005F0001F93CF93DF9314B815B8189B06C0199BAF
:1006000002C08DE003C08BE001C08AE0809300014E
:1006100081E887B98FEF88B98BE184B981E085B92A
:100620008EE38AB9579A87EF8BB984B7877F84BFE7
:10063000809160008861809360001092600080ED7E
:1006400097E09093D6048093D5041092750510928C
:10065000740510925208109251081092730510926E
:1006600072051092710510927005809100018A3018
:1006700011F4289801C0289A0E94920E0E942A071D
:100680000E94F2180E94F00E0E94F0170E940B3E8A
:1006900078941092360786E48093370788E0809339
:1006A000380781E08093390720910001822F6AE0AA
:1006B0000E940F45492F50E0822F0E940F4590E085
:1006C00024E630E03F932F9326E430E03F932F93CE
:1006D0001F921F925F934F939F938F938AE691E0AF
:1006E0009F938F931F920E94E70989E491E09F9363
:1006F0008F931F920E94E7098DB79EB740960FB661
:10070000F8949EBF0FBE8DBF809100018C3010F415
:10071000299A01C02998A1E0B0E00E94B645802D39
:100720008734A9F18AE191E09F938F931F920E94F1
:10073000E7090E941228C0E0D0E00F900F900F90C0
:100740009BE7E92E98E0F92E1C2FC23039F0C33018
:1007500019F40E94B92604C0C43010F00E94642726
:1007600043E5B701812F0E94C8022196C630D1050A
:1007700059F783E022E030E0D901082E0E94BE45FF
:1007800087E421503040D901082E0E94BE45C4E0C4
:10079000D0E0DE010E94B645802D853050F081E02A
:1007A00091E09F938F931F920E94E7090F900F9003
:1007B0000F902297DE010E94B645802D863028F0EA
:1007C00082E0DE01082E0E94BE4543E56BE778E03B
:1007D0000E94E202DE010E94B645802D863028F09C
:1007E00082E0DE01082E0E94BE4590E09F938F9329
:1007F00086EE90E09F938F931F920E94E70980916D
:1008000083080F900F900F900F900F9080FD03C002
:10081000C8EED3E020C089EC90E09F938F931F92A5
:100820000E94E70988EE93E00E94610DEC010E94AE
:1008300075120F900F900F90CE010E946A0D8823C1
:10084000D9F384EC90E09F938F931F920E94E70965
:100850000F900F900F900E940F25809100018A3019
:1008600011F4289801C0289A80ED97E09093D6045F
:100870008093D50485E58093480786EB90E09F93AD
:100880008F931F920E94E709809183080F900F9029
:100890000F9082FF03C08AEA90E002C082EA90E0F3
:1008A0009F938F931F920E94E7090F900F900F90D4
:1008B0008EE990E09F938F931F920E94E7090E9418
:1008C000BE1288E893E190938F0380938E0381E0BA
:1008D000809347070F900F900F908091D204882348
:1008E00009F4A5C01092D20480914607882319F01C
:1008F0000E94950202C00E94BE280E944B232091B4
:1009000000012A3011F4289801C0289A809105012D
:10091000882321F081508093050112C01092C404F5
:100920001092C504109252071092920510929105F0
:1009300010929405109293051092960510929505C9
:1009400080916F05882329F080916F0581508093F5
:100950006F0580918E0390918F03892B01F585E0BF
:1009600090E090938F0380938E030E94CC18809127
:100970000803909109038F5F9F4FF9F480917805E8
:100980008823D9F080E197E29093D6048093D50430
:1009900080E890E090930903809308030EC0809153
:1009A0008E0390918F03019790938F0380938E0312
:1009B0002A3011F4289801C0289A8091D204882303
:1009C00021F080917805882311F40E944D070E9440
:1009D0004608CE010E946A0D882339F120910E034A
:1009E00030910F038091930890E0281739079CF409
:1009F00080910803909109038F5F9F4F61F480E716
:100A000097E19093D6048093D50480E093E090938F
:100A10000903809308030E94E53F84E08093D70494
:100A200084E190E00E94610DEC010E94B74080914A
:100A3000D704882309F051CF0E9426404ECF1F9241
:100A40000F920FB60F9211248F939F93EF93FF9302
:100A5000809103018823E1F48091CE049091CF042A
:100A600001969093CF048093CE04FC01E85FF94F88
:100A7000E081ED3019F08639910539F41092CF04F8
:100A80001092CE0481E080930301E093C60004C07D
:100A90001092CF041092CE04FF91EF919F918F910D
:100AA0000F900FBE0F901F9018951F920F920FB6C8
:100AB0000F9211242F933F934F938F939F93AF9354
:100AC000BF93CF93DF93EF93FF938091C600809302
:100AD000B8044091C904463910F01092C8048091BE
:100AE000B8048D3009F05CC08091C804823009F0F0
:100AF00057C01092C804A42FB0E0FD01ED5AF84F82
:100B00003081ED01CC5AD84F28818091CC0490914E
:100B1000CD04831B9109821B91099F709093CD0492
:100B20008093CC049C0196E0369527959A95E1F741
:100B3000235C2093CB04982F9F73935C9093CA04FB
:100B40008081281729F48881981711F491E006C054
:100B50008091BB048F5F8093BB0490E08091B904C7
:100B6000882309F065C0992309F462C081E080936D
:100B7000B9044093BC04AB5AB84F8DE08C9380917C
:100B80005707823509F054C088E190E02CE00FB699
:100B9000F894A895809360000FBE2093600048C031
:100BA0008091C8048130D9F0813018F08230F1F59D
:100BB00021C08091B804833239F48091B90488232C
:100BC00019F481E08093C8048091B804809355079C
:100BD00081E08093C9048091B80490E022C082E053
:100BE0008093C804E42FF0E08091B804EB5AF84FEA
:100BF000808309C0E42FF0E08091B804EB5AF84FED
:100C00008083463920F44F5F4093C90402C010929C
:100C1000C8042091B8048091CC049091CD04820F37
:100C2000911D9093CD048093CC0402C01092C8040F
:100C3000FF91EF91DF91CF91BF91AF919F918F91F4
:100C40004F913F912F910F900FBE0F901F901895CD
:100C5000DC0120E030E040E050E008C0FA01E85F4D
:100C6000F94F8081280F311D4F5F5F4F4A175B0797
:100C7000A9F73F70C90136E0969587953A95E1F757
:100C8000835CFD01E85FF94F808311962F73235C2D
:100C9000FD01E85FF94F2083A75FB94F8DE08C938A
:100CA00010920301809108068093C60008951F9357
:100CB000CF93DF93EA01722F93E29093080660933B
:100CC000090680930A06A3E0B0E060E04FC0FE0191
:100CD000E60FF11D90816F5F715019F410E040E054
:100CE0000FC0FE01E60FF11D40816F5F715011F4DE
:100CF00010E006C0FE01E60FF11D10816F5F71501C
:100D0000892F86958695835CFD01E85FF94F808386
:100D100050E09A0184E0369527958A95E1F7892F6E
:100D200090E083709070F4E0880F991FFA95E1F7D6
:100D3000282B235CFD01E75FF94F2083812F8295EB
:100D40008695869583704F705070440F551F440FE1
:100D5000551F842B835CFD01E65FF94F80831F7371
:100D6000135CFD01E55FF94F10831496772309F0BA
:100D7000AECFCD010E942806DF91CF911F9108953B
:100D80001F93CF93DF93EC0170E0A22FB0E0129796
:100D900048C0E42FF0E0EB5AF84F30814F5FE42F6A
:100DA000F0E0EB5AF84F50814F5FE42FF0E0EB5A40
:100DB000F84F10814F5FE42FF0E0EB5AF84F20819D
:100DC0004F5F842F90E0A817B90774F15D53FE01BF
:100DD000E70FF11D852F82958F703D53330F330F31
:100DE000382B3083613001F1912F9D537F5FFE01DD
:100DF000E70FF11D71505295507F892F869586958A
:100E0000582B508363506F3F79F07E5FFE01E70FF0
:100E1000F11D9295990F990F907C2D53922B9083F1
:100E20007F5F662309F0B5CFDF91CF911F910895C1
:100E30001F93182F8A3019F48DE00E9418078091B3
:100E4000C00085FFFCCF1093C60080E090E01F91AA
:100E500008950895E1ECF0E088E18083A0ECB0E033
:100E60008C9182608C938081806880838081806493
:100E700080838AE28093C40088EC90E00E94610D38
:100E800090933507809334078CED90E00E94610DBC
:100E9000909354078093530708958091030188230A
:100EA00009F4F3C08091B404882371F080910301A8
:100EB000882351F0609107062BE048E457E087E46F
:100EC0000E9457061092B4048091530790915407E2
:100ED0000E946A0D882309F448C080910301882389
:100EE00009F443C06091200570912105809122058D
:100EF000909123052CE630E040E050E00E946445EC
:100F0000309341072093400760912805709129058F
:100F100080912A0590912B052CE630E040E050E0CE
:100F20000E946445309343072093420780918705D0
:100F30008093440780918805809345076091070658
:100F400028E040E457E087E70E9457068091460773
:100F5000853018F086E08093460783E690E00E9493
:100F6000610D9093540780935307809134079091BB
:100F700035070E946A0D882321F48091B6048823E6
:100F8000B1F080910301882391F06091070622E47B
:100F90004BEE57E084E40E9457061092B6048AEFA5
:100FA00090E00E94610D9093350780933407609123
:100FB00004016F3F89F0462F50E094E0440F551F25
:100FC0009A95E1F74A5F5E4F605D20E181E40E94FF
:100FD00057068FEF8093040190912D089923A1F07B
:100FE00080910301882381F083E280930806909327
:100FF00009068DE080930A061092030110922D08D5
:10100000809108068093C6008091B504882359F129
:1010100080910301882339F10E94C7121092B50410
:101020003091BE04932F9F5F9093BE04943021F0C3
:101030008091BF04882359F026E14DE458E060E038
:1010400084E30E9457068FEF8093BE040CC044E1F6
:10105000949FA00111244D5D5C4F24E160E0832F3B
:101060008F5C0E9457068091B704882371F08091AD
:101070000301882351F0609107062AE046E357E018
:1010800086E50E9457061092B70408951F93CF93E8
:10109000DF93CDB7DEB724970FB6F894DEBF0FBE4F
:1010A000CDBF8091B904882309F42EC180915707E0
:1010B000883609F486C0893690F4823609F453C024
:1010C000833630F48B34F1F0813609F01BC13FC018
:1010D000833609F45FC0873609F014C1A5C0813793
:1010E00038F48C3608F0D0C08B3609F00BC18DC0B7
:1010F000843709F481C0863709F492C0813709F03A
:1011000001C196C02091BC0443E062E0CE0101968B
:101110000E94C00689819A8190935D0580935C0549
:1011200080915C0590915D0520915E0530915F0591
:10113000845E9D4F821B930B68E671E00E942F45F1
:10114000845B90409093610580936005DBC02091A3
:10115000BC0443E062E0CE0103960E94C0068B818E
:101160008093040113C02091BC0443E06BE088E449
:1011700097E00E94C0068091010590914A07892B53
:10118000809301058091510780932D088FEF809304
:101190000501B8C02091BC0443E06BE088E497E00F
:1011A0000E94C0068091010590914A07892B809387
:1011B00001058091510780932D0881E08093B6044A
:1011C000E5CF2091BC0443E062E0CE0103960E948B
:1011D000C006809101059B81892B809301058C813C
:1011E0008F3F21F481E08093BF0402C01092BF04BE
:1011F00081E08093B50486C02091BC0443E064E0A4
:1012000080EC94E00E94C006C1CF2091BC0443E072
:1012100064E084EC94E00E94C0068091C704B4CFDF
:1012200081E08093B7046EC081E08093B4046AC00B
:101230002091BC0443E062E0CE0103960E94C00608
:10124000809103018823E1F38B818F3F89F0863001
:1012500010F085E08B8343E56BE778E08B810E949B
:10126000E202609107068B8123E54BE758E008C056
:10127000109107060E94860223E54BE758E0612F94
:10128000855B0E9457063EC02091BC0443E063E5A5
:101290008BE798E00E94C0068091570743E56BE713
:1012A00078E08B560E94C802809157078B56A2E0C7
:1012B000B0E0082E0E94BE456091A60870E080E074
:1012C00090E024EC39E040E050E00E94F04460936C
:1012D000920370939303809394039093950360918A
:1012E000A70870E080E090E00E94F04460939603CD
:1012F0007093970380939803909399030E948602BA
:101300000E94A4261092B90424960FB6F894DEBF6A
:101310000FBECDBFDF91CF911F910895982F80917F
:101320002E08813069F480910005E82FF0E0ED5D32
:10133000FC4F90838F5F8093000521E030E005C073
:10134000892F0E941807282F30E0C90108951F93A4
:10135000182F04C080E30E948E0911501116D4F397
:101360001F9108951F93182F04C080E20E948E09D8
:1013700011501116D4F31F9108950F931F93CF931B
:10138000DF938C01EB0108C0F8010F5F1F4FE49160
:101390008E2F0E948E0921972097B1F7DF91CF9170
:1013A0001F910F9108950F931F93CF93DF938C019B
:1013B000EB0106C0F80181918F010E948E092197EF
:1013C0002097C1F7DF91CF911F910F9108952F9230
:1013D0003F924F925F926F927F928F929F92AF92C5
:1013E000BF92CF92DF92EF92FF920F931F93CF9312
:1013F000DF93CDB7DEB7E5970FB6F894DEBF0FBE2B
:10140000CDBF2B968FAD2B9780932E08CE01835B9B
:101410009F4F9B838A832D964EAC5FAC2D971EA663
:101420001FA618AA19AA9E01225D3F4F3DAB2CAB07
:10143000820102C00F5F1F4FF801F490FF2019F0E6
:10144000F5E2FF16B9F7B8016419750919F0C20180
:101450000E94BD09FF2009F445C228010894411CDF
:10146000511C1982AA81BB8133241BAA2FEF2AABFE
:10147000F2010894411C511CB490632D70E061701E
:10148000707035E7B31621F08B2D80628837C9F470
:101490006115710559F02D913D914D915C91139716
:1014A0002EA73FA748AB59AB14960BC08D919C91CA
:1014B00011979C0140E050E02EA73FA748AB59ABE5
:1014C000129630E2B31621F48981882389F61CC074
:1014D00043E2B41611F458E055C08AE2B81621F080
:1014E0009DE2B91671F408C0FD011296E081EBABE4
:1014F000E7FFBECFE195EBABE0E13E2AFFED3F22F7
:10150000B7CF2BE2B21611F4B982B2CF3EE2B316D6
:1015100099F5F2010894411C511C84918A3221F002
:10152000B82E20E030E01DC0FD01129640815181AF
:1015300057FF02C04FEF5FEF4AAB9ACFC90153E0AC
:10154000880F991F5A95E1F7220F331F280F391F73
:101550002B0D311D20533040F2010894411C511CC9
:10156000B4908B2D80538A3048F3A90137FF02C015
:101570004FEF5FEF4AAB85CF40E3B41629F434FC5C
:1015800077CF50E2352A74CF8B2D81538930D8F430
:1015900020E030E0C90103E0880F991F0A95E1F7C8
:1015A000220F331F280F391F2B0D311D20533040C0
:1015B000F2010894411C511CB4908B2D80538A3049
:1015C00048F32BAB5ECF88E6B81619F494E0392ABD
:1015D0004FCFECE6BE1619F4F1E03F2A49CFBB83AA
:1015E000AA8323E6B21639F41296BB83AA83129714
:1015F0008C918E8322C134E4B31639F044E6B416DC
:1016000031F059E6B516A9F502C081E0382A30FE5E
:1016100008C01496BB83AA835E914E913E912E9191
:101620000AC01296BB83AA839E918E919C01442787
:1016300037FD4095542F2EA73FA748AB59AB8EA539
:101640009FA5A8A9B9A9BB238CF42EA53FA548A99D
:1016500059A950954095309521953F4F4F4F5F4F79
:101660002EA73FA748AB59AB8DE28983BAE02B2E5A
:1016700080C03FE4B31621F04FE6B41631F402C047
:1016800051E0352AA8E02A2E73C080E7B81689F405
:101690001296BB83AA839E918E919C0140E050E0FC
:1016A0002EA73FA748AB59AB30E4332AF8E7BF2E4B
:1016B0005DC043E7B416D1F51296BB83AA83DE90D2
:1016C000CE90C114D10489F488E28E838EE68F8394
:1016D00085E788878CE689878A8789E28B871C86DD
:1016E000E6E0CE2ED12CCC0EDD1E5AA957FD14C03B
:1016F000452F552747FD509560E070E0C6010E94D8
:10170000C842009711F4FAA80EC0F82EFC188AA956
:101710008F154CF4F82E07C0F60101900020E9F770
:101720003197FE2EFC18198240E090C095E5B9165D
:1017300021F0A5E7BA1631F402C0B1E03B2A7AE005
:10174000272E16C0E8E5BE1621F0F8E7BF1609F00F
:1017500070C033FE0BC02EA53FA548A959A921157D
:1017600031054105510511F030E4332A60E1262EA0
:1017700019824AA947FD02C05FED35228EA59FA5BB
:10178000A8A9B9A90097A105B10549F49AA9992377
:1017900031F45EE2C52ED12CCC0EDD1E46C06EA407
:1017A0007FA488A899A84EE2C42ED12CCC0EDD1EB1
:1017B000E22CFF2400E010E06EA57FA588A999A97E
:1017C000A80197010E9442456A3020F430E3A32E1D
:1017D000A60E08C027E5A22EA60EA8E5BA1611F49B
:1017E000BFEDAB22F601A2926F016EA57FA588A97D
:1017F00099A9A80197010E9442452EA73FA748AB8F
:1018000059AB6E147F048006910618F039014A0125
:10181000D3CFF8E02F1649F433FE07C020E3A21619
:1018200021F080E3D6018E936D01FCA8FC184AA933
:101830000DC0BB2009F456C0BE82198296E0C92EA5
:10184000D12CCC0EDD1E40E0FF24F394E42EEF18E3
:10185000E7FCEE248981882319F08F2D8F5F06C065
:1018600036FC02C08F2D02C08F2D8E5FA82EAE0CCD
:10187000032D10E080E3882E912C80229122811488
:10188000910421F48BA98A190E94B20989818823C5
:1018900029F061E070E0CE01019609C006FF09C0A1
:1018A00080E38C83BD8262E070E0CE0104960E94EA
:1018B000D309B0E28B16910421F48BA98A190E94F6
:1018C000A7098E2D0E94A7096F2D772767FD7095B8
:1018D000C6010E94D30904FFABCD8BA98A190E94CF
:1018E000B209A6CDE5960FB6F894DEBF0FBECDBF08
:1018F000DF91CF911F910F91FF90EF90DF90CF90EC
:10190000BF90AF909F908F907F906F905F904F901F
:101910003F902F9008951F920F920FB60F921124AF
:101920002F933F935F936F937F938F939F93AF9387
:10193000BF938091D704882329F08091D7048150E8
:101940008093D7048091DA0481508093DA048F3F2A
:10195000B9F489E08093DA0480910D038F5F817080
:1019600080930D03882319F481E08093D204809141
:10197000D0049091D10401969093D1048093D00427
:101980008091D5049091D6040297B8F08091D50447
:101990009091D60401979093D6048093D5048091BA
:1019A000D5049091D6042091080330910903822335
:1019B0009323892B09F071C006C08FEF9FEF90939E
:1019C000090380930803809100018A3039F404C030
:1019D0005A9A05C0479A03C05A9801C04798809107
:1019E000830883FF60C0349B0AC08091D304909128
:1019F000D40401969093D4048093D30454C080916E
:101A0000D3049091D404892B69F18091D3049091EF
:101A1000D4048A56914030F52091D3043091D404F7
:101A20008091D3049091D40469E270E00E941B4538
:101A3000260F371F3093D4042093D3048091D3040E
:101A40009091D4040B9750F08091D3049091D404DA
:101A50000A9790935D0580935C0504C010925D0524
:101A600010925C0580915C0590915D0520915E056A
:101A700030915F05845E9D4F821B930B68E671E099
:101A80000E942F45845B9040909361058093600590
:101A90001092D4041092D30406C0809100018A30C1
:101AA00009F098CF95CFBF91AF919F918F917F9182
:101AB0006F915F913F912F910F900FBE0F901F90EC
:101AC00018952091D0043091D1042F5F3F4F820FA1
:101AD000931F08952091D0043091D104821B930B61
:101AE000892F99278695807490E008951F920F9210
:101AF0000FB60F9211248F939F93809106039091BC
:101B00000703892B11F05F9A01C05F9883E08093EF
:101B1000B000809170008E7F809370009F918F91B4
:101B20000F900FBE0F901F9018951F920F920FB637
:101B30000F9211242F933F934F935F936F937F9353
:101B40008F939F93AF93BF93CF93DF93EF93FF93C5
:101B50008091060390910703049709F085C0809156
:101B6000A70390E0880F991F40910A0350910B033F
:101B70009A01220F331F240F351F820F931F64E039
:101B800070E00E942F4570930B0360930A03EB01F2
:101B9000E096D093D904C093D8048091BD08609199
:101BA0009D082091200530912105409122055091FA
:101BB000230580FF0EC070E080E090E00E94F044BA
:101BC00020E030E440E050E00E946445C20FD31FA3
:101BD0000DC070E080E090E00E94F04420E030E42E
:101BE00040E050E00E946445C21BD30BD093D9045F
:101BF000C093D8042091D8043091D90480919E08D4
:101C000043E0849FC00111242817390740F08091D8
:101C10009F08849FC00111248217930720F490939A
:101C2000D9048093D8042091D8043091D9043093FA
:101C3000160820931508C9016FEF70E00E941B453C
:101C40008D9740F4235B3F4F3093D9042093D80401
:101C500083E101C080E680930C038091D8048095D5
:101C60008093B30083EC40C08091060390910703FA
:101C7000892B39F18091060390910703049708F5A9
:101C80002091D8043091D9042F3F310561F058F0EC
:101C90005F9A83E08093B0002F5F30403093D90487
:101CA0002093D80423C083E88093B00080910C0374
:101CB0008093B30081E090E0909307038093060344
:101CC00015C08091060390910703892B79F48091C8
:101CD000A00890E0880F991F880F991F9093070321
:101CE000809306035F9883E08093B00080910603A1
:101CF0009091070301979093070380930603FF9148
:101D0000EF91DF91CF91BF91AF919F918F917F9193
:101D10006F915F914F913F912F910F900FBE0F9058
:101D20001F9018958091D0049091D1040B969093B8
:101D3000DC048093DB0482E085BD83EA84BD17BCAC
:101D400088E788BD86E086BD83EC8093B00084E0A0
:101D50008093B100E0E7F0E0808182608083EEE66E
:101D6000F0E08081816080838AE08093B3001092EC
:101D7000B2000895AC012091D0043091D1042F5FBE
:101D80003F4F03C08FEE80937A008091D0049091F2
:101D9000D104B901681B790BCB01840F951F8070AA
:101DA0009078892F99278695882361F30895AC014F
:101DB0002091D0043091D1042F5F3F4F8091D00407
:101DC0009091D104B901681B790BCB01840F951F49
:101DD00080709078892F99278695882379F30895C4
:101DE00010927C008FEE80937A0008951F920F92DC
:101DF0000FB60F921124EF92FF920F931F932F9320
:101E00003F934F935F936F937F938F939F93AF9382
:101E1000BF93EF93FF9310927A008091FC048F5F41
:101E20008093FC048150853009F486C0863090F49C
:101E3000823009F440C0833030F48823F1F08130DF
:101E400009F076C22FC0833009F441C0843009F014
:101E50006FC25AC0883009F4C2C0893038F4863065
:101E600009F483C0873009F063C29CC0893009F44B
:101E7000D3C08A3009F05CC2C6C1809178009091CD
:101E800079009093FB048093FA0481E08093FD0431
:101E90008091F1049091F20401969093F204809362
:101EA000F1044AC280917800909179009093F904EE
:101EB0008093F80492C0809178009091790090937B
:101EC000F7048093F60484E08093FD0435C24091CA
:101ED0000E0350910F0380917800909179009A0140
:101EE000220F331F240F351F63E070E00E941B4553
:101EF000260F371F369527953695279530930F0374
:101F000020930E0386E0E0CF209178003091790095
:101F10008091160590911705821B930B90933008C2
:101F200080932F0880912F08909130089093E404BB
:101F30008093E30487E0C8CF809178009091790086
:101F40002091140530911505821B930B90933B084B
:101F500080933A0880913A0890913B089093E60468
:101F60008093E5041092FD04E7C180910001209167
:101F7000FA043091FB048A3049F480917800909102
:101F80007900820F931F9695879506C080917800FF
:101F900090917900820F931F9093E2048093E10463
:101FA00081E092CF809100012091F8043091F904F2
:101FB0008A3049F48091780090917900820F931FC4
:101FC0009695879506C08091780090917900820F50
:101FD000931F9093E0048093DF0482E075CF80919B
:101FE00000012091F6043091F7048A3049F4809181
:101FF000780090917900820F931F9695879506C07F
:102000008091780090917900820F931F9093DE0465
:102010008093DD0485E058CF60917800709179005D
:10202000E0901A05F0901B0500911C0510911D050C
:10203000882777FD8095982F0E94D543A8019701A6
:102040000E94D5420E94A2437093E8046093E70483
:102050008091E7049091E80402970CF43EC06091EF
:102060001A0570911B0580911C0590911D0520E0BB
:1020700030E84BE354E40E94104488230CF078C00D
:1020800060911A0570911B0580911C0590911D05AA
:102090002AE037ED43EA5CE30E94D64260931A05DA
:1020A00070931B0580931C0590931D0580919B05E3
:1020B00090919C05845F914008F05AC060911A0588
:1020C00070911B0580911C0590911D052DEC3CEC39
:1020D0004CEC5DE30E94D64243C08091E7049091AE
:1020E000E8048F5F9F4F0CF043C060911A05709118
:1020F0001B0580911C0590911D0520E030E849E00A
:1021000054E40E94144418169CF560911A057091CD
:102110001B0580911C0590911D052AE037ED43EACF
:102120005CE30E94D54260931A0570931B0580936F
:102130001C0590931D0580919B0590919C05845FE3
:102140009140B0F460911A0570911B0580911C05B7
:1021500090911D052DEC3CEC4CEC5DE30E94D542CA
:1021600060931A0570931B0580931C0590931D05C1
:1021700081E08093EE0480917800909179009093B3
:1021800032088093310820915805309159054091CB
:102190005A0550915B058091E7049091E804AA27C5
:1021A00097FDA095BA2F820F931FA41FB51F809390
:1021B000580590935905A0935A05B0935B05E0909C
:1021C0005805F090590500915A0510915B056091F2
:1021D00058057091590580915A0590915B0520E052
:1021E00034E040E050E00E946445E21AF30A040B38
:1021F000150BE0925805F092590500935A0510937B
:102200005B0583E061CE80913F089091400820916A
:10221000780030917900820F931F9093400880934B
:102220003F08809137088F5F809337088091370887
:10223000853008F47DC0809178009091790090936A
:10224000150380931403109237084091EF045091C6
:10225000F004209133083091340880913F08909128
:102260004008281B390B8091790590917A05281B2D
:10227000390B80919E0390E0BC01269FC001279FEF
:10228000900D369F900D11249A0163E0220F331FA9
:102290006A95E1F7241B350B820F931F68E070E00D
:1022A0000E942F457093F0046093EF0420913F0843
:1022B00030914008E0901003F09011030091120358
:1022C00010911303C801B701660F771F881F991F6C
:1022D0006E0D7F1D801F911F442737FD4095542FA1
:1022E000620F731F841F951F24E030E040E050E030
:1022F0000E9464452093100330931103409312030E
:1023000050931303209133083091340880911003C7
:1023100090911103A0911203B0911303281B390B64
:1023200030937A05209379051092400810923F0867
:102330001092FD041092FC048091FD0480937C00B7
:102340008091FC04882319F08FEE80937A00FF912E
:10235000EF91BF91AF919F918F917F916F915F911D
:102360004F913F912F911F910F91FF90EF900F9000
:102370000FBE0F901F9018950F931F931092F304A8
:102380001092F4041092F5040CE810E0133019F4E4
:102390000B3008F009E08091DD049091DE048C5F41
:1023A000934024F48091160381500CC08091DD0489
:1023B0009091DE048750944014F411E006C080919F
:1023C00016038F5F8093160310E08091DF049091D5
:1023D000E0048C5F934024F48091170381500AC07D
:1023E0008091DF049091E0048750944034F0809114
:1023F00017038F5F8093170301C01F5F8091E10473
:102400009091E2048C5F934024F4809118038150F2
:102410000AC08091E1049091E2048750944034F026
:10242000809118038F5F8093180301C01F5F88E0BD
:10243000809303050E94F617809116038A3030F4CA
:1024400081E08093F3048AE0809316038091160361
:10245000863F30F081E08093F30485EF809316038C
:10246000809117038A3030F481E08093F4048AE08D
:102470008093170380911703863F30F081E08093AB
:10248000F40485EF80931703809118038A3030F4A9
:1024900081E08093F5048AE080931803809118030B
:1024A000863F30F081E08093F50485EF8093180338
:1024B000809103058823E1F7109237088FEE80930F
:1024C0007A00809137088823E1F30A3020F48AE00B
:1024D00090E00E94BA0E015009F058CF86E490E0D7
:1024E0000E94BA0E1F910F9108950F931F93CF93DF
:1024F000DF93A3E0B0E00E94B645802DC82FD0E066
:10250000C531D10508F02A97C7BD84E690E00E9446
:10251000BA0E809114039091150382559340C8F42C
:10252000C0E0D0E016C0C7BD82E390E00E94BA0EC2
:102530001F930F931F920E94E709809114039091BB
:1025400015030F900F900F908458934038F0219608
:1025500002C00EE911E0CA3FD10528F3A3E0B0E0C4
:102560000C2E0E94BE45C0933C088CE291E00E9474
:10257000BA0EDF91CF911F910F910895E3E2F3E03E
:1025800080E2819383E0E337F807D1F708951F9342
:1025900080910105282F30E0C90181709070682F6B
:1025A0008823A9F080910205882311F0815002C090
:1025B0008091730380930205E3E2F3E080E281936C
:1025C00043E0E337F407D1F78FEF8093BE04A9010E
:1025D0004270507021FF10C0809102058F5F809380
:1025E0000205E3E2F3E080E2819383E0E337F8075A
:1025F000D1F78FEF8093BE04662321F0452B11F0B5
:102600001092020580910205282F30E08A3040F4B4
:1026100081E1809300053F932F9389EC94E007C0FC
:1026200080E1809300053F932F9384EC94E09F9387
:102630008F9381E08F930E94E7090F900F900F9086
:102640000F900F9010910205153009F405C2163055
:1026500090F4123009F4C9C0133030F4112309F199
:10266000113009F0B4C465C0133009F414C114303A
:1026700009F0ADC46DC1183009F48DC3193038F4B8
:10268000163009F40DC3173009F0A1C460C31A3025
:1026900009F404C41A3008F4BDC31B3009F097C410
:1026A0003FC41092000584EB94E09F938F9311E058
:1026B0001F930E94E70984E18093000520910001A7
:1026C000822F6AE00E940F45492F50E0822F0E941E
:1026D0000F4590E024E630E03F932F9326E430E06E
:1026E0003F932F931F921F925F934F939F938F93CC
:1026F0008FE994E09F938F931F930E94E70988E2EC
:10270000809300050E94860290E09F938F9382E958
:1027100094E09F938F931F930E94E7098CE380932B
:10272000000582E894E09F938F931F930E94E7092E
:1027300009C38091830880FF3AC010920005809100
:10274000790590917A059F938F9383E794E09F9307
:102750008F931F930E94E70984E180930005809185
:102760007B0590917C059F938F9384E694E09F93E3
:102770008F931F930E94E70988E280930005809160
:102780001403909115039F938F9385E594E09F9395
:102790008F931F930E94E7098CE38093000580913B
:1027A0003C0890E09F938F9386E494E06EC384E1AD
:1027B000809300058FE394E09F938F931F930E9473
:1027C000E70988E28093000581E394E09F938F936B
:1027D0001F930E94E7094DB75EB74A5F5F4F0FB680
:1027E000F8945EBF0FBE4DBFF7C31092000587E29D
:1027F00094E09F938F9311E01F930E94E70984E177
:10280000809300056091200570912105809122053B
:102810009091230520E034E040E050E00E946445C0
:102820005F934F933F932F9388E194E09F938F930F
:102830001F930E94E70988E28093000560912805B4
:102840007091290580912A0590912B0520E034E0B4
:1028500040E050E00E9464455F934F933F932F9375
:1028600089E094E09F938F931F930E94E7098CE384
:102870008093000580915C0590915D059F938F93F7
:102880008AEF93E09F938F931F930E94E7098DB780
:102890009EB7469696C3109200058091510890917C
:1028A000520820914F08309150089F938F933F9387
:1028B0002F938AEE93E09F938F9311E01F930E94D2
:1028C000E70984E1809300058091550890915608AE
:1028D00020915308309154089F938F933F932F93E7
:1028E0008AED93E09F938F931F930E94E70988E2FC
:1028F000809300058091590890915A0820915708BB
:10290000309158089F938F933F932F938AEC93E0D5
:102910009F938F931F930E94E7098CE38093000598
:1029200080915D0890915E0820915B0830915C0871
:102930009F938F933F932F938AEB93E09F938F9373
:102940001F930E94E7094DB75EB7445E5F4F47CFC4
:1029500010920005E0917C08F0E0EE0FFF1FE35BB2
:10296000F74F20813181E0917B08F0E0EE0FFF1FEF
:10297000E35BF74F808191813F932F939F938F93D8
:102980008AEA93E09F938F9311E01F930E94E709D7
:1029900084E180930005E0917E08F0E0EE0FFF1FD8
:1029A000E35BF74F20813181E0917D08F0E0EE0F8D
:1029B000FF1FE35BF74F808191813F932F939F939C
:1029C0008F938AE993E09F938F931F930E94E70967
:1029D00088E280930005E0918008F0E0EE0FFF1F91
:1029E000E35BF74F20813181E0917F08F0E0EE0F4B
:1029F000FF1FE35BF74F808191813F932F939F935C
:102A00008F938AE893E09F938F931F930E94E70927
:102A10008CE380930005E0918208F0E0EE0FFF1F49
:102A2000E35BF74F20813181E0918108F0E0EE0F08
:102A3000FF1FE35BF74F808191813F932F939F931B
:102A40008F938AE793E09F938F931F930E94E709E8
:102A50008DB79EB74C96B5C2109200058CE693E0F8
:102A60009F938F9311E01F930E94E70980910001CB
:102A70000F900F900F908A3009F04DC084E1809341
:102A8000000520910A0530910B058091DD0490919D
:102A9000DE04821B930B3F932F939F938F938DE5BF
:102AA00093E09F938F931F930E94E70988E280939E
:102AB000000520910C0530910D058091DF04909167
:102AC000E004821B930B3F932F939F938F938EE48D
:102AD00093E09F938F931F930E94E7098CE3809369
:102AE000000520910E0530910F058091E104909131
:102AF000E204A901481B590B3F932F935F934F9317
:102B00008FE393E09F938F931F930E94E7098DB704
:102B10009EB7459656C2E0910A05F0910B058B30A1
:102B200009F058C084E180930005CF0162E070E0B5
:102B30000E942F458091DD049091DE048E1B9F0B37
:102B40007F936F939F938F9380E393E09F938F93F3
:102B50001F930E94E70988E28093000520910C05ED
:102B600030910D05C90162E070E00E942F4580910F
:102B7000DF049091E004821B930B7F936F939F93EC
:102B80008F9381E293E09F938F931F930E94E709B5
:102B90008CE38093000520910E0530910F05C9014B
:102BA00062E070E00E942F458091E1049091E20480
:102BB000281B390B7F936F933F932F9382E193E010
:102BC0009F938F931F930E94E7094DB75EB74B5EAB
:102BD0005F4F05CE84E1809300052091160330E01D
:102BE000CF0162E070E00E942F458091DD0490915A
:102BF000DE048E1B9F0B3F932F937F936F939F93C6
:102C00008F938EEF92E09F938F931F930E94E7091B
:102C100088E2809300052091170330E0E0910C05D5
:102C2000F0910D05CF0162E070E00E942F45809188
:102C3000DF049091E0048E1B9F0B3F932F937F93B3
:102C40006F939F938F938AEE92E09F938F931F933E
:102C50000E94E7098CE380930005E0911803F0E0FF
:102C600020910E0530910F05C90162E070E00E94CD
:102C70002F458091E1049091E204281B390BFF93CA
:102C8000EF937F936F933F932F9386ED92E09F9303
:102C90008F931F930E94E7098DB79EB74B9691C102
:102CA0001092000589EC92E09F938F9311E01F939F
:102CB0000E94E70984E180930005809114059091BA
:102CC00015052091E5043091E6049F938F933F937F
:102CD0002F938AEB92E09F938F931F930E94E709B3
:102CE00088E2809300058091160590911705209148
:102CF000E3043091E4049F938F933F932F938BEAE7
:102D000092E09F938F931F930E94E7098CE3809337
:102D1000000560911A0570911B0580911C0590912A
:102D20001D050E94A2432091E5083091E6087F939B
:102D30006F933F932F938CE992E09F938F931F9310
:102D40000E94E7094DB75EB7485E5F4F48CD84E10A
:102D50008093000580910E0390910F039F938F93B2
:102D60008DE892E09F938F9311E01F930E94E709F3
:102D700088E28093000580916F0590E09F938F9388
:102D80008EE792E09F938F931F930E94E7098DB780
:102D90009EB70A9616C1109200058FE692E09F93A7
:102DA0008F9311E01F930E94E70984E1809300054F
:102DB00080916005909161059F938F9380E692E0EA
:102DC0009F938F931F930E94E70988E280930005E9
:102DD00080915C0590915D059F938F9381E592E0D2
:102DE0009F938F931F930E94E7098CE380930005C4
:102DF00080915E0590915F059F938F9382E492E0AE
:102E00009F938F931F930E94E7094DB75EB74E5E65
:102E10005F4FE5CC109200058091670590916805A1
:102E20009F938F9386E392E09F938F9311E01F937C
:102E30000E94E70984E180930005809169059091E3
:102E40006A059F938F938AE292E09F938F931F93DB
:102E50000E94E70988E28093000580916B059091BC
:102E60006C059F938F938EE192E09F938F931F93B6
:102E70000E94E7098CE38093000580916D05909195
:102E80006E059F938F9382E192E09F938F931F93A0
:102E90000E94E7098DB79EB7449693C01092000533
:102EA0008AE092E09F938F9311E01F930E94E709BD
:102EB00084E1809300058091A70390E09F938F9316
:102EC0008CEF91E09F938F931F930E94E70988E214
:102ED000809300058091D8049091D9049F938F939B
:102EE0008EEE91E09F938F931F930E94E7098CE3EE
:102EF0008093000520919F0830E080919E0890E02B
:102F00003F932F939F938F9380EE91E09F938F93A6
:102F10001F930E94E7094DB75EB74C5E5F4F5FCCD1
:102F20001092000580ED91E09F938F9311E01F9325
:102F30000E94E70984E18093000520914C07332724
:102F400027FD309580914B07992787FD90953F93FA
:102F50002F939F938F9380EC91E09F938F931F9378
:102F60000E94E70988E28093000520914D073327EE
:102F700027FD309580914E0790E03F932F939F93CC
:102F80008F9380EB91E09F938F931F930E94E709AB
:102F90008CE3809300052091520730E080914F0729
:102FA000992787FD90953F932F939F938F9380EA66
:102FB00091E09F938F931F930E94E7098DB79EB76F
:102FC00048960FB6F8949EBF0FBE8DBF05C0115036
:102FD0001093730310920205109201051F9108953A
:102FE0001092B9008AE28093B800089585EA809330
:102FF000BC0080E090E0089584E98093BC000895CF
:103000001092B9008093BB0085E88093BC0080E0FB
:1030100090E008951F920F920FB60F9211248F9394
:103020009F93EF93FF93809103058F5F8093030538
:103030008150E82FF0E0E731F10508F09FC0E85C2F
:10304000FF4FEE0FFF1F0590F491E02D0994809142
:103050000405880F8E5A29C0809104058F5F8093E4
:10306000040581508230B1F0833030F4882361F060
:10307000813009F083C00BC0843091F0843068F057
:10308000853009F07BC00FC08091E7080EC08091A9
:10309000DD080BC08091160908C08091D90805C0D1
:1030A0008091FB0802C08091FD081092B9008093C6
:1030B000BB0085E88093BC0061C084E98093BC00BC
:1030C00080910405863018F4109203053BC01092DD
:1030D000040538C080910505880F8D5AE6CF85EC30
:1030E000E9CF8091BB00E0910505F0E0EF5BF74F81
:1030F0008083DFCF809105059091BB00E82FF0E041
:10310000EF5BF74F96838F5F80930505863058F10C
:103110001092050528C01092B90080E1C8CF8091B7
:103120001603C3CF1092B90082E1C1CF809117037B
:10313000BCCF84E98093BC008AE090E090938F0339
:1031400080938E0385EAB6CF1092B90088E9AFCF9D
:103150001092B90084E1ABCF80911803A6CF1092F2
:10316000B90080E8A4CF84E98093BC008AE090E0B5
:1031700090938F0380938E03109203058091BC007F
:1031800080688093BC00FF91EF919F918F910F9089
:103190000FBE0F901F9018954CEB50E084E9DA01B8
:1031A0008C93109203052BEB30E0F9018081109293
:1031B000040580E88C931092BD001092BA00108232
:1031C000E9EBF0E01082A8EBB0E01C9210828AE2FA
:1031D0008C9385EADA018C931082F901108285E8DC
:1031E0008C93089583EC80938100EFE6F0E080817A
:1031F0008062808310920F0510920E0510920D05CB
:1032000010920C0510920B0510920A0508951F925A
:103210000F920FB60F9211240F931F932F933F938A
:103220004F935F936F937F938F939F93AF93BF93CE
:10323000CF93DF93EF93FF93209186003091870027
:103240008091080590910905281B390B8091860013
:10325000909187009093090580930805C9018D54CA
:1032600094400091060510910705835F9A4160F430
:103270000430110514F01092740381E090E09093F3
:103280000705809306058AC00A3011050CF086C038
:10329000C9018B5F9040845B914008F068C0E901F0
:1032A000C25DD140F801EE0FFF1FE35BF74F808155
:1032B00091819E01281B390BC90137FF03C09095EE
:1032C00081959F4F06974CF480916F05883C28F4B8
:1032D00080916F05865F80936F05F801EE0FFF1FE9
:1032E000E35BF74F20813181C901880F991F820F5D
:1032F000931F8C0F9D1F64E070E00E942F459B017F
:10330000CE010196861797071CF42150304006C065
:1033100021976C177D0714F42F5F3F4F80916F0545
:10332000E801CC0FDD1F833CB8F0FE01E35BF74FF3
:1033300080819181A901481B590BCA0163E070E0AB
:103340000E942F45CB01880F991F860F971FCD59DB
:10335000D74F9983888304C0CD59D74F19821882DB
:10336000F801EE0FFF1FE35BF74F31832083F80175
:103370003196F0930705E0930605E530F10511F469
:103380005D9A06C05D98E630F10511F45C9A05C0BF
:103390005C98379711F45B9A01C05B98FF91EF91AD
:1033A000DF91CF91BF91AF919F918F917F916F915D
:1033B0005F914F913F912F911F910F910F900FBEF1
:1033C0000F901F9018952F923F924F925F926F929D
:1033D0007F928F929F92AF92BF92CF92DF92EF92A5
:1033E000FF920F931F93CF93DF93CDB7DEB726974E
:1033F0000FB6F894DEBF0FBECDBF2091E10430912F
:10340000E20480910E0590910F05821B930B90931F
:103410000509809304092091E1043091E204809130
:10342000F5089091F608821B930B90937A0880938D
:1034300079088091DF049091E00420910C0530918F
:103440000D05821B930B9093D1088093D008809137
:10345000DD049091DE0420910A0530910B05821B5A
:10346000930B9093DC088093DB086091E5047091E6
:10347000E604882777FD8095982F2CE030E040E027
:1034800050E00E94F0449B01AC01609100097091F2
:103490000109882777FD8095982F620F731F841F7D
:1034A000951F22E030E040E050E00E9464453093F8
:1034B0000109209300096091E3047091E4048827D6
:1034C00077FD8095982F2CE030E040E050E00E949E
:1034D000F0449B01AC016091120970911309882797
:1034E00077FD8095982F620F731F841F951F22E030
:1034F00030E040E050E00E9464453093130920938F
:1035000012096091E7047091E804882777FD80959F
:10351000982F2091E5083091E608442737FD409523
:10352000542F620F731F841F951F22E030E040E08C
:1035300050E00E9464453093E6082093E50820910E
:10354000E5043091E604C901880F991F820F931F8B
:10355000880F991F880F991FAA2797FDA095BA2F4A
:10356000209130053091310540913205509133055D
:10357000280F391F4A1F5B1F2093300530933105F8
:1035800040933205509333052091E3043091E404D5
:10359000C901880F991F820F931F880F991F880FE9
:1035A000991FAA2797FDA095BA2F20913405309135
:1035B00035054091360550913705280F391F4A1FB0
:1035C0005B1F2093340530933505409336055093A7
:1035D00037052091E5043091E6048091EE08909142
:1035E000EF08820F931F9093EF088093EE082091CD
:1035F000E3043091E4048091070990910809820F57
:10360000931F909308098093070980911805909162
:10361000190501969093190580931805E0903108DB
:10362000F0903208A0901A05B0901B05C0901C05C0
:10363000D0901D05609138057091390580913A054B
:1036400090913B050E94D5433B014C010027F7FCBC
:103650000095102FC801B7010E94D543A60195011E
:103660000E94D5429B01AC01C401B3010E94D64225
:103670000E94A243609338057093390580933A0500
:1036800090933B0580910409909105099C01442782
:1036900037FD4095542F80910E0990910F09A0910C
:1036A0001009B0911109280F391F4A1F5B1F209381
:1036B0000E0930930F09409310095093110980911E
:1036C0000409909105093C01882477FC8094982C8A
:1036D0008091500590915105A0915205B0915305EC
:1036E000680E791E8A1E9B1E6092500570925105CD
:1036F0008092520590925305203B83E8380788E07A
:10370000480780E0580764F0205B33484840504049
:1037100020930E0930930F0940931009509311091B
:1037200080910E0990910F09A0911009B091110993
:10373000B7FF0CC080559C47A74FBF4F80930E0921
:1037400090930F09A0931009B0931109E09181059E
:10375000EE83EE2309F08AC080918205882309F068
:1037600085C08091830886FF81C06091790870913F
:103770007A08E0908F05FF2400E010E0882777FDAD
:103780008095982F20914005309141054091420548
:10379000509143050E94F04420E038E040E050E0C2
:1037A0000E946445CA01B901A80197010E94F04432
:1037B00020E030E140E050E00E94644559016A0198
:1037C0002093E1053093E2054093E3055093E4052F
:1037D0006091790870917A08882777FD8095982FF5
:1037E000209148053091490540914A0550914B057B
:1037F0000E94F04420E038E040E050E00E94644540
:10380000CA01B901A80197010E94F04420E030E10B
:1038100040E050E00E9464452093DD053093DE05D2
:103820004093DF055093E005D601C501D7FE07C0E0
:10383000B095A095909581959F4FAF4FBF4F813820
:103840009105A105B10574F457FF07C05095409547
:10385000309521953F4F4F4F5F4F2138310541053E
:103860005105A4F081E08093640510C01092DD053D
:103870001092DE051092DF051092E0051092E1052E
:103880001092E2051092E3051092E4058091D008B1
:103890009091D1082091E1053091E2054091E30536
:1038A0005091E4052A833B834C835D83820F931FF1
:1038B0009093D1088093D0080091D0081091D1083E
:1038C000A090DD05B090DE05C090DF05D090E0054A
:1038D00080919005282E332444245524C201B1013F
:1038E000A60195010E94F04420E032E040E050E063
:1038F0000E946445020F131F1093D1080093D00853
:103900002091D0083091D108442737FD4095542F9D
:1039100080914C0590914D05A0914E05B0914F05B9
:10392000820F931FA41FB51F80934C0590934D05E4
:10393000A0934E05B0934F058091D0089091D10887
:1039400020917D0530917E05821B930BAA2797FD60
:10395000A095BA2F209148053091490540914A051C
:1039600050914B05820F931FA41FB51F80934805EC
:1039700090934905A0934A05B0934B05E0909603B8
:10398000F09097030091980310919903E816F906B7
:103990000A071B07C4F488EA91E6A0E0B0E08E199C
:1039A0009F09A00BB10B8093480590934905A09304
:1039B0004A05B0934B0580934C0590934D05A09319
:1039C0004E05B0934F0522273327A9012E193F0931
:1039D000400B510B8091480590914905A0914A05F3
:1039E000B0914B0582179307A407B507B4F4D8012B
:1039F000C701885A9146A040B040809348059093F3
:103A00004905A0934A05B0934B0580934C059093CC
:103A10004D05A0934E05B0934F058091DF04909122
:103A2000E0040F9734F488E19CEF9093D1088093E1
:103A3000D0088091DF049091E004079734F480E38C
:103A400098EF9093D1088093D0083091000139838A
:103A50003A30A9F48091DF049091E004835F9340B1
:103A600034F088EE93E09093D1088093D008809151
:103A7000DF049091E0048A5F9340DCF014C08091F1
:103A8000DF049091E004855E974034F088EE93E087
:103A90009093D1088093D0088091DF049091E00446
:103AA000835F974034F080ED97E09093D108809346
:103AB000D0088091DB089091DC088A199B099093CB
:103AC000DC088093DB080091DB081091DC08C20160
:103AD000B1012A813B814C815D810E94F04420E04C
:103AE00032E040E050E00E946445021B130B10934B
:103AF000DC080093DB082091DB083091DC084427C8
:103B000037FD4095542F8091440590914505A09133
:103B10004605B0914705820F931FA41FB51F8093E0
:103B2000440590934505A0934605B09347058091C1
:103B3000DB089091DC0820917F0530918005821B85
:103B4000930BAA2797FDA095BA2F2091400530919D
:103B500041054091420550914305820F931FA41FD8
:103B6000B51F8093400590934105A0934205B09303
:103B70004305E0909203F090930300919403109119
:103B80009503E816F9060A071B07C4F488EA91E6CC
:103B9000A0E0B0E08E199F09A00BB10B8093400507
:103BA00090934105A0934205B0934305809344054B
:103BB00090934505A0934605B093470522273327E8
:103BC000A9012E193F09400B510B8091400590919E
:103BD0004105A0914205B091430582179307A407C0
:103BE000B507B4F4D801C701885A9146A040B04047
:103BF0008093400590934105A0934205B0934305FF
:103C00008093440590934505A0934605B0934705DE
:103C10008091DD049091DE040F9734F488E19CEFED
:103C20009093DC088093DB088091DD049091DE04A2
:103C3000079734F480E398EF9093DC088093DB08D7
:103C400029812A30A9F48091DD049091DE04835FFC
:103C5000934034F088EE93E09093DC088093DB0887
:103C60008091DD049091DE048A5F9340DCF014C003
:103C70008091DD049091DE04855E974034F088EEFB
:103C800093E09093DC088093DB088091DD049091B1
:103C9000DE04835F974034F080ED97E09093DC087A
:103CA0008093DB088FEE80937A0060923C057092DF
:103CB0003D0580923E0590923F0580914005909190
:103CC0004105A0914205B091430580932005909352
:103CD0002105A0932205B09323058091480590917A
:103CE0004905A0914A05B0914B0580932805909312
:103CF0002905A0932A05B0932B0580914405909146
:103D00004505A0914605B091470580932405909301
:103D10002505A0932605B093270580914C05909129
:103D20004D05A0914E05B0914F0580932C059093C1
:103D30002D05A0932E05B0932F058091830887FF52
:103D400063C0FE81FF2309F05FC080918205882354
:103D500009F05AC08091DB089091DC08893C9105FC
:103D60005CF02091DB083091DC088091DB089091B9
:103D7000DC082052334011C08091DB089091DC08B0
:103D800088539F4FA4F42091DB083091DC08809188
:103D9000DB089091DC08205E3C4F880F991F880F4C
:103DA000991F280F391F3093DC082093DB0880917E
:103DB000D0089091D108893C91055CF02091D00801
:103DC0003091D1088091D0089091D1082052334091
:103DD00011C08091D0089091D10888539F4FA4F4CE
:103DE0002091D0083091D1088091D0089091D108CD
:103DF000205E3C4F880F991F880F991F280F391F8D
:103E00003093D1082093D008209167053091680540
:103E100080917F08E82FF0E0EE0FFF1FE35BF74F84
:103E20008081918182599F4F281739071CF42F5F99
:103E30003F4F0CC08081918182599F4F8217930719
:103E40004CF42115310531F0215030403093680594
:103E5000209367052091690530916A05809180085B
:103E6000E82FF0E0EE0FFF1FE35BF74F80819181B9
:103E700082599F4F281739071CF42F5F3F4F0CC002
:103E80008081918182599F4F821793074CF42115AD
:103E9000310531F02150304030936A052093690597
:103EA00020916B0530916C0580918108E82FF0E03E
:103EB000EE0FFF1FE35BF74F8081918182599F4F87
:103EC000281739071CF42F5F3F4F0CC08081918168
:103ED00082599F4F821793074CF42115310531F019
:103EE0002150304030936C0520936B0520916D0577
:103EF00030916E0580918208E82FF0E0EE0FFF1FF1
:103F0000E35BF74F8081918182599F4F28173907D2
:103F10001CF42F5F3F4F0CC08081918182599F4FCD
:103F2000821793074CF42115310531F021503040B0
:103F300030936E0520936D0580916705909168051B
:103F400097FF05C010926805109267050AC08F3F61
:103F5000910539F034F08FEF90E0909368058093ED
:103F600067058091690590916A0597FF05C01092D9
:103F70006A05109269050AC08F3F910539F034F047
:103F80008FEF90E090936A058093690580916B05AF
:103F900090916C0597FF05C010926C0510926B050F
:103FA0000AC08F3F910539F034F08FEF90E0909385
:103FB0006C0580936B0580916D0590916E0597FF60
:103FC00005C010926E0510926D050AC08F3F9105D5
:103FD00039F034F08FEF90E090936E0580936D058B
:103FE00026960FB6F894DEBF0FBECDBFDF91CF91FE
:103FF0001F910F91FF90EF90DF90CF90BF90AF9007
:104000009F908F907F906F905F904F903F902F90F8
:104010000895809186088B3F98F08B3F19F480912A
:1040200067050EC08C3F19F48091690509C08D3F6A
:1040300019F480916B0504C08E3F21F480916D05C9
:1040400080939F03809185088B3F98F08B3F19F4F4
:10405000809167050EC08C3F19F48091690509C0F5
:104060008D3F19F480916B0504C08E3F21F480913F
:104070006D0580939E0380919E03882319F410920E
:104080009E0305C0843618F084E680939E038091D9
:1040900087088B3F98F08B3F19F4809167050EC01D
:1040A0008C3F19F48091690509C08D3F19F4809106
:1040B0006B0504C08E3F21F480916D058093A003B1
:1040C0008091A003882319F41092A00305C08436C0
:1040D00018F084E68093A003809189088B3F98F0C4
:1040E0008B3F19F4809167050EC08C3F19F48091C5
:1040F000690509C08D3F19F480916B0504C08E3F9E
:1041000021F480916D058093A103809190088B3FED
:1041100098F08B3F19F4809167050EC08C3F19F41D
:104120008091690509C08D3F19F480916B0504C029
:104130008E3F21F480916D058093A20380919108B8
:104140008B3F98F08B3F19F4809167050EC08C3F30
:1041500019F48091690509C08D3F19F480916B05B0
:1041600004C08E3F21F480916D058093A30380915C
:10417000A3038B3010F48AE002C08F3F11F48093C8
:10418000A303809192088B3F98F08B3F19F48091A4
:1041900067050EC08C3F19F48091690509C08D3FF9
:1041A00019F480916B0504C08E3F21F480916D0558
:1041B0008093A403809197088B3F98F08B3F19F46C
:1041C000809167050EC08C3F19F48091690509C084
:1041D0008D3F19F480916B0504C08E3F21F48091CE
:1041E0006D058093A603809198088B3F98F08B3FD4
:1041F00019F4809167050EC08C3F19F48091690510
:1042000009C08D3F19F480916B0504C08E3F21F4E5
:1042100080916D0580938705809199088B3F98F078
:104220008B3F19F4809167050EC08C3F19F4809183
:10423000690509C08D3F19F480916B0504C08E3F5C
:1042400021F480916D058093880580919A088B3FB9
:1042500098F08B3F19F4809167050EC08C3F19F4DC
:104260008091690509C08D3F19F480916B0504C0E8
:104270008E3F21F480916D058093890580919B0884
:104280008B3F98F08B3F19F4809167050EC08C3FEF
:1042900019F48091690509C08D3F19F480916B056F
:1042A00004C08E3F21F480916D0580938A05809132
:1042B000AB088B3F98F08B3F19F4809167050EC0D7
:1042C0008C3F19F48091690509C08D3F19F48091E4
:1042D0006B0504C08E3F21F480916D0580938B05A2
:1042E0008091AC088B3F98F08B3F19F48091670563
:1042F0000EC08C3F19F48091690509C08D3F19F4F7
:1043000080916B0504C08E3F21F480916D058093F0
:104310008C058091AD088B3F98F08B3F19F480910C
:1043200067050EC08C3F19F48091690509C08D3F67
:1043300019F480916B0504C08E3F21F480916D05C6
:1043400080938D058091AE088B3F98F08B3F19F4D8
:10435000809167050EC08C3F19F48091690509C0F2
:104360008D3F19F480916B0504C08E3F21F480913C
:104370006D0580938E0580919C088B3F98F08B3F54
:1043800019F4809167050EC08C3F19F4809169057E
:1043900009C08D3F19F480916B0504C08E3F21F454
:1043A00080916D058093A7038091A1088B3F98F0C1
:1043B0008B3F19F4809167050EC08C3F19F48091F2
:1043C000690509C08D3F19F480916B0504C08E3FCB
:1043D00021F480916D058093A8038091A4088B3F00
:1043E00098F08B3F19F4809167050EC08C3F19F44B
:1043F0008091690509C08D3F19F480916B0504C057
:104400008E3F21F480916D0580938F058091A508E2
:104410008B3F98F08B3F19F4809167050EC08C3F5D
:1044200019F48091690509C08D3F19F480916B05DD
:1044300004C08E3F21F480916D058093900580919A
:10444000AA088B3F98F08B3F19F4809167050EC046
:104450008C3F19F48091690509C08D3F19F4809152
:104460006B0504C08E3F21F480916D058093A903F4
:104470008091B0088B3F98F08B3F19F480916705CD
:104480000EC08C3F19F48091690509C08D3F19F465
:1044900080916B0504C08E3F21F480916D0580935F
:1044A000F0088091F008823010F481E002C08F3F64
:1044B00011F48093F0088091B2088B3F98F08B3F05
:1044C00019F4809167050EC08C3F19F4809169053D
:1044D00009C08D3F19F480916B0504C08E3F21F413
:1044E00080916D058093020980910209823010F459
:1044F00081E002C08F3F11F4809302098091B308DC
:104500008B3F98F08B3F19F4809167050EC08C3F6C
:1045100019F48091690509C08D3F19F480916B05EC
:1045200004C08E3F21F480916D058093DA0880915C
:10453000B4088B3F98F08B3F19F4809167050EC04B
:104540008C3F19F48091690509C08D3F19F4809161
:104550006B0504C08E3F21F480916D058093140992
:104560008091B5088B3F98F08B3F19F480916705D7
:104570000EC08C3F19F48091690509C08D3F19F474
:1045800080916B0504C08E3F21F480916D0580936E
:10459000D2088091B6088B3F98F08B3F19F4809138
:1045A00067050EC08C3F19F48091690509C08D3FE5
:1045B00019F480916B0504C08E3F21F480916D0544
:1045C0008093DE088091B7088B3F98F08B3F19F4F9
:1045D000809167050EC08C3F19F48091690509C070
:1045E0008D3F19F480916B0504C08E3F21F48091BA
:1045F0006D05809318098091B8088B3F98F08B3F28
:1046000019F4809167050EC08C3F19F480916905FB
:1046100009C08D3F19F480916B0504C08E3F21F4D1
:1046200080916D058093E0088091BB088B3F98F0E6
:104630008B3F19F4809167050EC08C3F19F480916F
:10464000690509C08D3F19F480916B0504C08E3F48
:1046500021F480916D05809315096091A60370E0A7
:1046600080E090E00E94284127E137EB41ED58E3DC
:104670000E948D4460939A0370939B0380939C03E4
:1046800090939D0380918E088093030980918D08FB
:104690008093DF08089580917805882381F5109232
:1046A000D9081092DD081092E708109216091092AE
:1046B000FB081092FD088091C004882331F080939C
:1046C0001609809116098093E7088091C104882318
:1046D00031F08093DD088091DD088093D9088091C6
:1046E000C204882311F08093FD088091C3048823BD
:1046F00011F08093FB0880919D058C7F03C0809111
:104700009D05816080939D058091E70890E09093DE
:104710000208809301088091160990E090930408A4
:10472000809303088091D90890E0909306088093C5
:1047300005088091DD0890E09093080880930708B1
:104740008091FD0890E090930A0880930908809179
:10475000FB0890E090930C0880930B0810920305DF
:10476000109204050E94F6170895809100018D3083
:1047700010F00E94BC1110927A008091DD0490919B
:10478000DE049093DC088093DB088091DF04909135
:10479000E0049093D1088093D0088091E104909137
:1047A000E20490930509809304096091E5047091F7
:1047B000E604882777FD8095982F2CE030E040E0D4
:1047C00050E00E94F04470930109609300096091E9
:1047D000E3047091E404882777FD8095982F0E9468
:1047E000F04470931309609312098091E70490914B
:1047F000E8049093E6088093E5088FEE80937A00B2
:10480000209167053091680580917F08E82FF0E0DE
:10481000EE0FFF1FE35BF74F8081918182599F4F1D
:10482000281739071CF42F5F3F4F0CC080819181FE
:1048300082599F4F821793074CF42115310531F0AF
:104840002150304030936805209367052091690519
:1048500030916A0580918008E82FF0E0EE0FFF1F8D
:10486000E35BF74F8081918182599F4F2817390769
:104870001CF42F5F3F4F0CC08081918182599F4F64
:10488000821793074CF42115310531F02150304047
:1048900030936A052093690520916B0530916C0572
:1048A00080918108E82FF0E0EE0FFF1FE35BF74FE8
:1048B0008081918182599F4F281739071CF42F5FFF
:1048C0003F4F0CC08081918182599F4F821793077F
:1048D0004CF42115310531F02150304030936C05F6
:1048E00020936B0520916D0530916E0580918208B3
:1048F000E82FF0E0EE0FFF1FE35BF74F808191811F
:1049000082599F4F281739071CF42F5F3F4F0CC067
:104910008081918182599F4F821793074CF4211512
:10492000310531F02150304030936E0520936D05F4
:10493000809167059091680597FF05C01092680502
:10494000109267050AC08F3F910539F034F08FEF60
:1049500090E0909368058093670580916905909138
:104960006A0597FF05C010926A05109269050AC092
:104970008F3F910539F034F08FEF90E090936A0506
:104980008093690580916B0590916C0597FF05C038
:1049900010926C0510926B050AC08F3F910539F09B
:1049A00034F08FEF90E090936C0580936B058091CD
:1049B0006D0590916E0597FF05C010926E051092DF
:1049C0006D050AC08F3F910539F034F08FEF90E00C
:1049D00090936E0580936D056091A60870E080E06D
:1049E00090E024EC39E040E050E00E94F044609315
:1049F0009203709393038093940390939503609133
:104A0000A70870E080E090E00E94F0446093960375
:104A1000709397038093980390939903089510924D
:104A2000150510921405109217051092160580E0D6
:104A300090E0A0E0B0E080931A0590931B05A0934E
:104A40001C05B0931D0510920B0510920A051092DB
:104A50000D0510920C0510920F0510920E05109284
:104A6000F6081092F50810928F05109290050E949A
:104A7000B52384E690E00E94BA0E0E94B52380918F
:104A8000830880FF10C08091140390911503875B09
:104A9000934038F480911403909115038E5E9240F8
:104AA00010F40E9475124091DD045091DE04509381
:104AB0000B0540930A052091DF043091E004309308
:104AC0000D0520930C058091E1049091E2049093F0
:104AD0000F0580930E058091E1049091E20490937C
:104AE000F6088093F5083093110520931005509334
:104AF00013054093120544E050E0DA010E94B645E8
:104B0000802D853038F1809112099091130997FF1B
:104B100003C0909581959F4F6CE070E00E942F45F7
:104B20007093170560931605809100099091010913
:104B300097FF03C0909581959F4F6CE070E00E94B5
:104B40002F4570931505609314056091310870919D
:104B5000320839C0DA010E94B645802D4F5F5F4FA1
:104B6000DA010E94B645202D90E0982F8827820F09
:104B7000911D90931505809314054F5F5F4FDA01E7
:104B80000E94B645802D4F5F5F4FDA010E94B64507
:104B9000202D90E0982F8827820F911D9093170564
:104BA000809316054F5F5F4FDA010E94B645602D76
:104BB0004F5F5F4FDA010E94B645202D70E0762FDF
:104BC0006627620F711D882777FD8095982F0E94B8
:104BD000D54360931A0570931B0580931C05909331
:104BE0001D05109240051092410510924205109249
:104BF0004305109244051092450510924605109207
:104C00004705109248051092490510924A051092E6
:104C10004B0510924C0510924D0510924E051092C6
:104C20004F051092500510925105109252051092A6
:104C300053051092DC081092DB081092D1081092F4
:104C4000D008109205091092040984E690E00E94B1
:104C5000BA0E8091100390911103A0911203B091AC
:104C6000130390933408809333081092F004109249
:104C7000EF04109258051092590510925A0510929F
:104C80005B0580915C0590915D0590935F05809335
:104C90005E050E94E13D82E390E09093D60480930C
:104CA000D5046091A60870E080E090E024EC39E043
:104CB00040E050E00E94F0446856754C8F4F9F4F83
:104CC000609392037093930380939403909395035E
:104CD0006091A70870E080E090E00E94F044685680
:104CE000754C8F4F9F4F60939603709397038093FB
:104CF0009803909399031092AB031092AA036091CA
:104D00005C0570915D05882777FD8095982F2EE0D2
:104D100036E040E050E00E94F04460930E0970934A
:104D20000F09809310099093110910926605109253
:104D3000650581E0809301010E94A84080919D0556
:104D4000846080939D0508951F93182F0EC0809155
:104D50007805882361F484E690E09093D6048093EC
:104D6000D5048AEF90E00E94D70E115080F71F9172
:104D7000089581E080937B0882E080937C0893E033
:104D800090937D08E4E0E0937E0855E050937F081F
:104D900076E07093800887E08093810868E06093F4
:104DA000820888EE809383083EE1309384088BEF7D
:104DB000809386088AE08093870830938508309333
:104DC00089089093880860938A0890E190938B08F3
:104DD00070938C0860938D0886EE80938E083093D4
:104DE0008F0880E88093900844E64093910888E714
:104DF000809392088EE58093930883E280939408D1
:104E000084E18093950810929608909397081092E9
:104E100098081092990810929A0810929B08109284
:104E2000AB081092AC081092AD081092AE084093F7
:104E30009C0888E280939D081092BD0892E39093AD
:104E40009E0886E980939F085093A0089093A1083C
:104E50002AE52093A2089093A3081092BC082093FF
:104E6000A4085093A50885E58093A6088093A70819
:104E700080E28093A808E093A9089093AA088FE5A0
:104E80008093AF0883EF8093B1083093B0083093DC
:104E9000B2088DEF8093B3084093B4082093B5080F
:104EA0002093B6082093B7081092B8087093B908F9
:104EB0006093BA08A2ECB8E0E5E7F3E08CE001907B
:104EC0000D928150E1F7089581E080937B0882E0A4
:104ED00080937C0823E020937D08E4E0E0937E0843
:104EE00035E030937F0866E06093800887E0809328
:104EF000810858E05093820888E6809383089EE1F9
:104F0000909384088BEF809386088AE080938708CB
:104F10009093850890938908209388088CE080936B
:104F20008A0880E180938B0860938C0850938D08E9
:104F300086EE80938E0890938F0880E88093900887
:104F400080E58093910888E7809392088EE58093AE
:104F5000930883E2809394089093950810929608A2
:104F600040E2409397081092980810929908109286
:104F70009A0810929B081092AB081092AC081092FD
:104F8000AD081092AE0874E670939C0888E2809396
:104F90009D081092BD0892E390939E0886E9809345
:104FA0009F083093A0089093A1082AE52093A208B7
:104FB0009093A3081092BC082093A4083093A508EE
:104FC00085E58093A6088093A7084093A808E093FE
:104FD000A9088BE48093AA088FE58093AF0883EF3C
:104FE0008093B10884E18093B0088093B2088DEF7C
:104FF0008093B3087093B4082093B5082093B60843
:105000002093B7081092B8086093B9085093BA0873
:10501000A2ECB8E0EFE7F3E08CE001900D92815054
:10502000E1F7089581E080937B0882E080937C081B
:1050300083E080937D0864E060937E0845E04093C0
:105040007F08E6E0E093800887E08093810878E0BD
:105050007093820888E6809383089EE19093840889
:105060008BEF809386088AE0809387089093850869
:1050700090938908609388083FE030938A08909362
:105080008B088CE080938C0870938D0886EE80935B
:105090008E0890938F0880E88093900880E5809335
:1050A000910856E9509392088EE58093930883E225
:1050B00080939408909395081092960880E28093CC
:1050C0009708109298081092990810929A081092D6
:1050D0009B081092AB081092AC081092AD08109289
:1050E000AE0824E620939C0888E280939D081092E5
:1050F000BD0882E380939E0850939F084093A008C8
:105100008093A1089AE59093A2088093A308109237
:10511000BC089093A4084093A50885E58093A60851
:105120008093A70880E18093A8086093A908209342
:10513000AA088FE58093AF0883EF8093B10830937E
:10514000B0083093B2088DEF8093B3082093B40871
:105150009093B5089093B6089093B7081092B8084A
:10516000E093B9087093BA08A2ECB8E0E7E8F3E07E
:105170008CE001900D928150E1F708952F923F92BB
:105180004F925F926F927F928F929F92AF92BF9257
:10519000CF92DF92EF92FF920F931F93CF93DF9303
:1051A000CDB7DEB7E8970FB6F894DEBF0FBECDBF20
:1051B0000E94E319409100014C3010F4299A01C07B
:1051C000299820917605309177058091DF08682F26
:1051D00070E0665F7F4F7C8B6B8B6217730714F4F4
:1051E0003C8B2B8B80916F05843608F06AC08091D0
:1051F0000501882399F480910803909109038F5F3A
:105200009F4F61F488E99AE39093D6048093D50484
:1052100080E09CE090930903809308038091BF0590
:105220009091C005009731F001979093C00580934D
:10523000BF0504C010927805109262054A3011F43F
:10524000289A01C0289880919B0590919C05895EC1
:105250009340A0F180919408E82FF0E0FC8BEB8B59
:1052600081E080936205A0917B08B0E0AA0FBB1F8C
:10527000FD01ED59F74F11821082E0917C082E2F2D
:1052800030E0220F331FC9018D59974FFC01118265
:105290001082A35BB74F11961C921E92235B374F6F
:1052A000D90111961C921E92E0917E08F0E0EE0F5B
:1052B000FF1FE35BF74F118210829EC210927805A8
:1052C0009BC280916F058D3808F496C210926205DA
:1052D0008091950822E3829FC00111249093C0051C
:1052E0008093BF05EB89FC89B9978CF08091780594
:1052F000882369F080919B0590919C05FFEF8F3F7B
:105300009F0729F0019690939C0580939B058091BF
:105310009B0590919C058F3F910509F038F51092FF
:10532000D9051092DA051092DB051092DC05109277
:10533000D5051092D6051092D7051092D8058A3F50
:105340009105C9F481E08093B8051092D1051092BF
:10535000D2051092D3051092D405109250051092E8
:105360005105109252051092530505C080919D057C
:10537000826080939D05E0917D08F0E0EE0FFF1FB5
:10538000E35BF74F80819181813591050CF487C1F2
:1053900080917805882309F082C180917E08E82FEA
:1053A000F0E0EE0FFF1FE35BF74F808191818C34BB
:1053B00091050CF4E7C08091BE058F5F8093BE0518
:1053C000893C08F46CC14C3010F4299801C0299A2A
:1053D000109278051092BE0510929C0510929B05C4
:1053E00080917B08282F30E0F901EE0FFF1FE35B6F
:1053F000F74F80819181873491059CF4E0917C087E
:10540000F0E0EE0FFF1FE35BF74F0190F081E02D1E
:10541000F7FF03C0F095E195FF4FE734F1050CF479
:105420006CC080917C08682F70E0DB01AA0FBB1F65
:10543000A35BB74F8D919C911197873491053CF0F8
:10544000F901EE0FFF1FE35BF74F808191818D9192
:105450009C918734910564F0F901EE0FFF1FE35B27
:10546000F74F808191818734910514F042E001C0AB
:1054700041E0FB01EE0FFF1FE35BF74F808191815D
:10548000863491055CF4F901EE0FFF1FE35BF74FE3
:1054900080819181873491050CF043E0FB01EE0F90
:1054A000FF1FE35BF74F808191818A5B9F4F5CF424
:1054B000F901EE0FFF1FE35BF74F80819181873485
:1054C00091050CF044E0660F771F635B774FDB01BB
:1054D0008D919C918A5B9F4F5CF4220F331F235B5D
:1054E000374FF90180819181863491050CF445E0B4
:1054F000A2E0B0E0042E0E94BE45E0917C08F0E0FE
:10550000EE0FFF1FE35BF74F0190F081E02DF7FFF7
:1055100003C0F095E195FF4F7497B4F4E0917B08D8
:10552000F0E0EE0FFF1FE35BF74F808191818A5B14
:105530009F4F54F481E08093460788EE93E0909368
:10554000D6048093D504ABC00E94860243E56BE786
:1055500078E00E94E2028091830880FF10C0809171
:10556000140390911503875B934038F480911403E2
:10557000909115038E5E924010F40E9475120E9465
:105580000F2586C080819181855B9F4F0CF085C07F
:105590008091BE058F5F8093BE05893C08F47FC073
:1055A0004C3010F4299801C0299A8FEF04E010E0E4
:1055B000D801082E0E94BE45109278051092BE05B3
:1055C00010929C0510929B050E940F258091140556
:1055D0009091150560E071E00E942F45D801062EDC
:1055E0000E94BE45809114059091150560E071E020
:1055F0000E942F450F5F1F4FD801082E0E94BE4505
:10560000809116059091170560E071E00E942F458A
:105610000F5F1F4FD801062E0E94BE4580911605D0
:105620009091170560E071E00E942F450F5F1F4FBA
:10563000D801082E0E94BE4560911A0570911B0585
:1056400080911C0590911D050E94A243DC01CB01B5
:1056500060E071E00E942F450F5F1F4FD801062EBA
:105660000E94BE4560911A0570911B0580911C0532
:1056700090911D050E94A243DC01CB0160E071E026
:105680000E942F450F5F1F4FD801082E0E94BE4574
:105690000E9486020E94A42602C01092BE05E091DC
:1056A0007D08F0E0EE0FFF1FE35BF74F80819181F3
:1056B0008B5A9F4F0CF0A0C080917E08482F50E07D
:1056C000FA01EE0FFF1FE35BF74F80819181855B4D
:1056D0009F4F0CF072C08091BD058F5F8093BD0518
:1056E000893C08F46CC088EC8093BD0581E090E0B3
:1056F00090939C0580939B0581E0809378051092A0
:10570000D1051092D2051092D3051092D4051092B3
:1057100050051092510510925205109253051092A7
:105720005405109255051092560510925705109287
:1057300040051092410510924205109243051092C7
:1057400048051092490510924A0510924B05809128
:10575000200590912105A0912205B0912305809309
:10576000440590934505A0934605B0934705809165
:10577000280590912905A0912A05B0912B058093C9
:105780004C0590934D05A0934E05B0934F05109294
:10579000D9051092DA051092DB051092DC05109203
:1057A000D5051092D6051092D7051092D805809194
:1057B0009D05886080939D0502C01092BD05440F31
:1057C000551F435B574FDA018D919C918C349105A5
:1057D0008CF08091BC058F5F8093BC05893C60F0A4
:1057E0001092780588EC8093BC0510929C0510926D
:1057F0009B0502C01092BC05809174038150809378
:105800007403809174038F3F29F08091620588238F
:1058100009F493C30E94092080917B08A82EBB2421
:10582000D501AA0FBB1FFD01E35BF74F208131813A
:1058300080918A08282E3324AD59B74FED91FC9101
:1058400000918B0810E0229DC001239D900D329D98
:10585000900D11244091AE055091AF059A01220F91
:10586000331F240F351F820F931F64E070E00E94E6
:105870002F454B01E09FC001E19F900DF09F900DDF
:105880001124880E991E9092AF058092AE05E0918A
:10589000E505F091E605FEABEDAB2091E905309111
:1058A000EA053CAB2BAB80917C08482F50E058AF09
:1058B0004FABFA01EE0FFF1FDF01A35BB74F8D91D6
:1058C0009C91ED59F74F0190F081E02DBC01629D54
:1058D000C001639D900D729D900D11244091AC0507
:1058E0005091AD059A01220F331F240F351F820FEF
:1058F000931F64E070E00E942F456B01E09FC001A0
:10590000E19F900DF09F900D1124C80ED91ED092EA
:10591000AD05C092AC058091E7059091E8059AAB82
:1059200089ABA091EB05B091EC05B8ABAFA7E091C6
:105930007E08AE2FB0E0AA0FBB1FA35BB74F0D9040
:10594000BC91A02DBEA7ADA7E0917D08F0E0EE0FC1
:10595000FF1FE35BF74F60807180E8E7F0E06E0EB9
:105960007F1E70927705609276056091A30370E0C8
:1059700080E090E00E94284120E030E040E251E4E5
:105980000E94D64220E030E040E85CE30E948D4473
:1059900069A77AA78BA79CA76093090970930A0946
:1059A00080930B0990930C096091A40370E080E050
:1059B00090E00E94284120E030EE4BE256E40E9445
:1059C0003A436093F7087093F8088093F90890932E
:1059D000FA082091C504222331F08AE090E09093E8
:1059E000D6048093D504E22F22FF09C080911509C7
:1059F000482F50E0440F551F440F551F10C023FD82
:105A000003C040E050E00BC08091150990E0880F82
:105A1000991F880F991F44275527481B590B209120
:105A2000910530919205C901F3E0880F991FFA950D
:105A3000E1F7821B930B840F951F68E070E00E94D2
:105A40002F452B017093920560939105E4FF09C0E7
:105A500080911509482F50E0440F551F440F551FE2
:105A600010C0E5FD03C040E050E00BC08091150977
:105A700090E0880F991F880F991F44275527481BCE
:105A8000590B80919305909194059C0163E0220F3E
:105A9000331F6A95E1F7281B390BCA01820F931F48
:105AA00068E070E00E942F457B017093940560933D
:105AB00093058091C404282F83FF03C082E390E004
:105AC00004C082FF07C08EEC9FEF909396058093F1
:105AD000950504C0109296051092950521FF09C006
:105AE0008091AA039091AB0301969093AB038093AE
:105AF000AA0324FF09C08091AA039091AB030197E8
:105B00009093AB038093AA0384012DA93EA9021BA5
:105B1000130B4BA95CA9041B150BC20162E070E0DA
:105B20000E942F45060F171F1093710500937005F3
:105B300069A97AA9C61AD70A8FA598A9C81AD90A35
:105B4000C70162E070E00E942F45C60ED71ED092BA
:105B50007305C09272052091950530919605220F2C
:105B6000331F220F331FADA5BEA52A1B3B0B30935D
:105B70007505209374058091520780FF54C0809171
:105B80001509813808F44FC080914B07992787FD8C
:105B90009095FC01E29DC001E39D900DF29D900D5A
:105BA0001124080F191F109371050093700580913F
:105BB0004C07992787FD9095AC01429DC001439DFC
:105BC000900D529D900D1124C80ED91ED0927305D0
:105BD000C092720580914D07992787FD9095280FF7
:105BE000391F30937505209374052091880830E0A3
:105BF00080914F07992787FD9095BC01269FC00192
:105C0000279F900D369F900D11249093AB038093A6
:105C1000AA0380914E0790E08615970524F490938F
:105C2000770580937605809176059091770597FFAB
:105C300004C010927705109276058091830882FF48
:105C40000CC080E090E0A0E0B0E08093F708909373
:105C5000F808A093F908B093FA0820E030E040E09B
:105C600050E069A57AA58BA59CA50E9410448823C5
:105C700064F480E090E0A0E0B0E0809309099093A4
:105C80000A09A0930B09B0930C0920E030E040E032
:105C900050E06091F7087091F8088091F9089091B0
:105CA000FA080E941044882364F480E090E0A0E0A9
:105CB000B0E08093F7089093F808A093F908B093A8
:105CC000FA08E0917005F0917105209197053091E7
:105CD0009805CF0164E070E00E942F4577FF03C074
:105CE000709561957F4F26173707C4F4CF01F7FFF2
:105CF00003C0909581959F4F64E070E00E942F450E
:105D00007093980560939705653671056CF084E68D
:105D100090E0909398058093970506C021503040FD
:105D20003093980520939705E0917205F0917305E3
:105D30002091990530919A05CF0164E070E00E94AE
:105D40002F4577FF03C0709561957F4F2617370762
:105D5000C4F4CF01F7FF03C0909581959F4F64E095
:105D600070E00E942F4570939A05609399056536FF
:105D700071056CF084E690E090939A058093990504
:105D800006C02150304030939A05209399058091A8
:105D90006205882341F010929805109297051092A1
:105DA0009A0510929905EFA9F8ADEE0FFF1FE35B7E
:105DB000F74F208131818091A208482F50E042178F
:105DC000530744F48091BC0882FF04C081E08093B3
:105DD000830512C0EFA9F8ADEE0FFF1FE35BF74F8D
:105DE000208131818091A308DA01A81BB1092A170B
:105DF0003B0714F410928305EFA9F8ADEE0FFF1FD7
:105E0000E35BF74F8081918166277727641B750BD1
:105E10008617970744F48091BC0883FF04C081E093
:105E20008093840518C0809184058823A1F0EFA990
:105E3000F8ADEE0FFF1FE35BF74FF8AFEFAB20813C
:105E400031818091A30890E0841B950B8217930702
:105E500014F410928405F501EE0FFF1FE35BF74F7A
:105E6000808191814817590744F48091BC0880FFD4
:105E700004C081E08093860515C080918605882343
:105E800089F0F501EE0FFF1FE35BF74F20813181B1
:105E90008091A308DA01A81BB1092A173B0714F463
:105EA00010928605F501EE0FFF1FE35BF74F80812F
:105EB00091818617970744F48091BC0881FF04C044
:105EC00081E08093850517C080918505882399F02E
:105ED000AA0CBB1CEDE4F8E0AE0EBF1ED5012D915F
:105EE0003C918091A30890E0841B950B8217930747
:105EF00014F41092850580918305882321F4809104
:105F00008405882321F081E08093820502C01092ED
:105F1000820580918605882321F480918505882358
:105F200051F081E0809381051092820510928305E3
:105F30001092840502C01092810580918205882309
:105F400021F480918105882351F08091A10890E08F
:105F5000EB89FC898E179F0714F49C8B8B8BF09137
:105F60006205F983FF2341F11092750510927405C3
:105F700010927105109270051092730510927205BF
:105F800080E090E0A8ECBFE38093090990930A09B0
:105F9000A0930B09B0930C098BE09CEBA2E3BCE34C
:105FA0008093F7089093F808A093F908B093FA0843
:105FB00010928205109281052091200530912105D3
:105FC00040912205509123052A833B834C835D83B6
:105FD0008091EA089091EB08A091EC08B091ED084F
:105FE000820F931FA41FB51F8093EA089093EB08BC
:105FF000A093EC08B093ED08409128055091290535
:1060000060912A0570912B054E835F83688779879D
:106010008091F1089091F208A091F308B091F408F2
:10602000840F951FA61FB71F8093F1089093F20865
:10603000A093F308B093F4086091240570912505AE
:1060400080912605909127056DA37EA38FA398A725
:106050008091E1089091E208A091E308B091E408F2
:106060002DA13EA14FA158A5820F931FA41FB51FBC
:106070008093E1089093E208A093E308B093E408CA
:1060800040912C0550912D0560912E0570912F05A2
:1060900049A35AA36BA37CA38091D5089091D608FD
:1060A000A091D708B091D808840F951FA61FB71FDD
:1060B0008093D5089093D608A093D708B093D808BA
:1060C000509181055A87552329F4809182058823B0
:1060D00009F460C01092300510923105109232051B
:1060E0001092330510923405109235051092360542
:1060F000109237051092EA081092EB081092EC0803
:106100001092ED081092F1081092F2081092F30824
:106110001092F4081092E1081092E2081092E3083D
:106120001092E4081092D5081092D6081092D70861
:106130001092D8088091400590914105A0914205A8
:10614000B09143058093440590934505A09346057F
:10615000B09347058091480590914905A0914A0563
:10616000B0914B0580934C0590934D05A0934E053F
:10617000B0934F051092F2041092F1041092800532
:1061800010927F0510927E0510927D056A85662328
:1061900009F0F3C080918205882309F0EEC0E090F9
:1061A0008F08FF2400E010E06A817B818C819D8153
:1061B000A80197010E94644559016A018091000974
:1061C00090910109AA2797FDA095BA2FA81AB90A9C
:1061D000CA0ADB0A6E817F8188859985A8019701AB
:1061E0000E94644579018A018091120990911309F6
:1061F000AA2797FDA095BA2FE81AF90A0A0B1B0BDC
:10620000C601B50120E130E040E050E00E94644565
:1062100059016A01C801B70120E130E040E050E0D7
:106220000E94644579018A018091970590919805B3
:10623000813491053CF48091990590919A058134BF
:106240009105A4F0C601B50123E030E040E050E044
:106250000E94644559016A01C801B70123E030E09A
:1062600040E050E00E94644579018A01E0917E0897
:10627000F0E0EE0FFF1FE35BF74F0190F081E02DA0
:10628000F7FF03C0F095E195FF4F7A97A4F0C601A0
:10629000B50123E030E040E050E00E946445590140
:1062A0006A01C801B70123E030E040E050E00E94FD
:1062B000644579018A0171E2A716B104C104D104D1
:1062C00034F070E2A72EB12CC12CD12C11C080EE7D
:1062D000A8168FEFB8068FEFC8068FEFD80644F4E4
:1062E00060EEA62E6FEFB62E6FEFC62E6FEFD62E96
:1062F00091E2E916F1040105110534F050E2E52EB2
:10630000F12C012D112D11C0A0EEEA16AFEFFA0607
:10631000AFEF0A07AFEF1A0744F440EEE42E4FEF59
:10632000F42E4FEF042F4FEF142F809140059091E2
:106330004105A0914205B09143058A199B09AC091A
:10634000BD098093400590934105A0934205B09309
:1063500043058091480590914905A0914A05B09167
:106360004B058E199F09A00BB10B809348059093A4
:106370004905A0934A05B0934B058091F104909193
:10638000F2048F3F910509F008F49CC4BA85BB2341
:1063900009F01AC480918205882309F015C4809100
:1063A0006405882309F010C46091EA087091EB0835
:1063B0008091EC089091ED0820E031E040E050E061
:1063C0000E94644519012A012093EA083093EB08E2
:1063D0004093EC085093ED086091F1087091F20839
:1063E0008091F3089091F40820E031E040E050E023
:1063F0000E9464452D8F3E8F4F8F58A32093F10844
:106400003093F2084093F3085093F408E0908F081B
:10641000FF2400E010E020913005309131054091DB
:10642000320550913305C801B7010E94F04420E0C5
:1064300031E040E050E00E94644559016A01209338
:106440003005309331054093320550933305209148
:106450003405309135054091360550913705C80116
:10646000B7010E94F04420E031E040E050E00E949B
:10647000644539014A012093340530933505409332
:106480003605509337056091380570913905809134
:106490003A0590913B0520E031E040E050E00E9459
:1064A0006445209338053093390540933A0550935D
:1064B0003B05E090A808FF2400E010E0C201B10114
:1064C0006A197B098C099D09A80197010E946445FE
:1064D0002093B4053093B5054093B6055093B705A6
:1064E000CA01B90120E031E040E050E00E9464457B
:1064F00069013093800520937F056D8D7E8D8F8D92
:1065000098A16619770988099909A80197010E943D
:106510006445CA01B90120E031E040E050E00E944A
:106520006445890130937E0520937D058091970510
:106530009091980581349105C4F4809199059091CA
:106540009A05813491058CF4E0917E08F0E0EE0F1D
:10655000FF1FE35BF74F0190F081E02DF7FF03C0D1
:10656000F095E195FF4F7A9794F0C60162E070E0F4
:106570000E942F457093800560937F05C80162E0FB
:1065800070E00E942F4570937E0560937D056091B9
:10659000E1087091E2088091E3089091E40820E01E
:1065A00031E040E050E00E9464452093E1083093E0
:1065B000E2084093E3085093E4086091D508709195
:1065C000D6088091D7089091D80820E031E040E0CB
:1065D00050E00E9464452093D5083093D60840933C
:1065E000D7085093D808EDA0FEA00FA118A52A81C6
:1065F0003B814C815D81E21AF30A040B150BE0929A
:10660000CD05F092CE050093CF051093D005A9A03B
:10661000BAA0CBA0DCA04E815F8168857985A41AE1
:10662000B50AC60AD70AA092C905B092CA05C09297
:10663000CB05D092CC05E092C505F092C60500933B
:10664000C7051093C805A092C105B092C205C092BB
:10665000C305D092C4058091440590914505A09151
:106660004605B09147058E199F09A00BB10B809389
:10667000440590934505A0934605B0934705809146
:106680004C0590914D05A0914E05B0914F058A198A
:106690009B09AC09BD0980934C0590934D05A093CF
:1066A0004E05B0934F052091650530916605213860
:1066B000310594F080910E0590910F05019690930D
:1066C0000F0580930E058091F5089091F6080196CC
:1066D0009093F6088093F50820583F4F94F48091EA
:1066E0000E0590910F05019790930F0580930E056D
:1066F0008091F5089091F60801979093F6088093A1
:10670000F5086D8D7E8D8F8D98A12AE130E040E0F7
:1067100050E00E94644530931A08209319081092A3
:1067200066051092650581E090E09093AB0580933B
:10673000AA058091A2059091A305A091A405B0910E
:10674000A50582199309A409B509815E914BAF4F44
:10675000BF4F8F539C49A040B04008F0C1C071E0CA
:10676000E71670E1F70670E0070770E017070CF412
:1067700052C08091A905882309F449C0D801C701F6
:106780002CE0B595A795979587952A95D1F7019611
:106790009093AB058093AA05D801C701F3E0B595A6
:1067A000A79597958795FA95D1F78093B40590931F
:1067B000B505A093B605B093B70589589341A0409D
:1067C000B04064F088E893E1A0E0B0E08093B405C5
:1067D0009093B505A093B605B093B7056091B40545
:1067E0007091B5058091B6059091B70520E031E034
:1067F00040E050E00E94644580917F0590918005C3
:10680000820F931F9093800580937F0566C081E07F
:106810008093A90562C01092A905F0E0EF16F0EF91
:10682000FF06FFEF0F07FFEF1F070CF056C0809128
:10683000A805882309F44DC088279927DC018E1903
:106840009F09A00BB10BECE0B595A795979587959F
:10685000EA95D1F701969093AB058093AA05C801FC
:10686000B70128E030E040E050E00E94644520930A
:10687000B4053093B5054093B6055093B705285736
:106880003C4E4F4F5F4F64F488E79CEEAFEFBFEF95
:106890008093B4059093B505A093B605B093B70562
:1068A0006091B4057091B5058091B6059091B705DA
:1068B00020E031E040E050E00E94644580917F0597
:1068C00090918005820F931F9093800580937F05A0
:1068D00011C081E08093A8050DC01092A8050AC0E0
:1068E0001092AB051092AA0588EE93E09093910365
:1068F000809390038091A908882E99248091AA05FD
:106900009091AB058816990624F49092AB0580927D
:10691000AA0571E0E71674E0F70670E0070770E07B
:10692000170774F080910A0590910B052091AA0534
:106930003091AB05820F931F90930B0580930A054E
:1069400080E0E8168CEFF8068FEF08078FEF180746
:1069500074F480910A0590910B052091AA0530915D
:10696000AB05821B930B90930B0580930A0581E086
:1069700090E09093AB058093AA051092B005109219
:10698000B1051092B2051092B30580919E059091C9
:106990009F05A091A005B091A1052D8D3E8D4F8D35
:1069A00058A1821B930BA40BB50B815E914BAF4F8B
:1069B000BF4F8F539C49A040B04008F0C1C041E098
:1069C000A41640E1B40640E0C40640E0D4060CF44E
:1069D00052C08091A705882309F449C0D601C5019A
:1069E0007CE0B595A795979587957A95D1F701960F
:1069F0009093AB058093AA05D601C50163E0B595D8
:106A0000A795979587956A95D1F78093B005909350
:106A1000B105A093B205B093B30589589341A04046
:106A2000B04064F088E893E1A0E0B0E08093B00566
:106A30009093B105A093B205B093B3056091B005F2
:106A40007091B1058091B2059091B30520E031E0DD
:106A500040E050E00E94644580917D0590917E0564
:106A6000820F931F90937E0580937D0566C081E021
:106A70008093A70562C01092A70560E0A61660EF9C
:106A8000B6066FEFC6066FEFD6060CF056C08091C3
:106A9000A605882309F44DC088279927DC018A19A7
:106AA0009B09AC09BD095CE0B595A79597958795BD
:106AB0005A95D1F701969093AB058093AA05C6012C
:106AC000B50128E030E040E050E00E9464452093AA
:106AD000B0053093B1054093B2055093B3052857E4
:106AE0003C4E4F4F5F4F64F488E79CEEAFEFBFEF33
:106AF0008093B0059093B105A093B205B093B30510
:106B00006091B0057091B1058091B2059091B30587
:106B100020E031E040E050E00E94644580917D0536
:106B200090917E05820F931F90937E0580937D0543
:106B300011C081E08093A6050DC01092A6050AC081
:106B40001092AB051092AA0588EE93E09093910302
:106B5000809390038091AA059091AB0588169906C1
:106B600024F49092AB058092AA0581E0A81684E0F7
:106B7000B80680E0C80680E0D80674F080910C0565
:106B800090910D052091AA053091AB05820F931FBE
:106B900090930D0580930C0590E0A9169CEFB90623
:106BA0009FEFC9069FEFD906CCF480910C05909118
:106BB0000D052091AA053091AB05821B930B909394
:106BC0000D0580930C050AC010927E0510927D057C
:106BD0001092800510927F051092640520E030E04D
:106BE00040E050E06091F7087091F8088091F90852
:106BF0009091FA080E941044882341F410927E0577
:106C000010927D051092800510927F058091EA0810
:106C10009091EB08A091EC08B091ED088093A2054B
:106C20009093A305A093A405B093A5058091F108C6
:106C30009091F208A091F308B091F40880939E051A
:106C400090939F05A093A005B093A10510923005E5
:106C500010923105109232051092330510923405CE
:106C600010923505109236051092370510923805AE
:106C70001092390510923A0510923B051092EA08DD
:106C80001092EB081092EC081092ED081092F108A7
:106C90001092F2081092F3081092F4081092E10892
:106CA0001092E2081092E3081092E4081092D508BE
:106CB0001092D6081092D7081092D8081092F204B9
:106CC0001092F104C0907405D09075058601D7FE2E
:106CD00004C0002711270C191D09003111056CF0A3
:106CE00088EE93E0909391038093900380918308C2
:106CF00084FD03C081E08093B805E0908C08B60164
:106D0000882777FD8095982F2E2D30E040E050E0C9
:106D10000E94F0449801442737FD4095542F0E946B
:106D2000F04420E032E040E050E00E9464458901F8
:106D30009A01FF24EC9CC001ED9C900DFC9C900DF1
:106D4000112464E070E00E942F45600F711F9B01C9
:106D5000442737FD4095542F298F3A8F4B8F5C8FF6
:106D60002093D1053093D2054093D3055093D40599
:106D70008091500590915105A0915205B091530515
:106D8000821B930BA40BB50B809350059093510578
:106D9000A0935205B09353058155934CA040B04049
:106DA00064F080E593ECA0E0B0E080935005909310
:106DB0005105A0935205B0935305809150059091D1
:106DC0005105A0915205B0915305805B9C43AF4F94
:106DD000BF4F64F480EB9CE3AFEFBFEF80935005AF
:106DE00090935105A0935205B093530580915C0593
:106DF00090915D05892B09F42EC18091830883FF52
:106E00002AC16A817B818C819D8120E032E040E053
:106E100050E00E946445890137FF03C01095019539
:106E20001F4F6E817F818885998520E032E040E0A8
:106E300050E00E946445190137FF04C0309421944A
:106E400031083394201631060CF41801E0905C05EB
:106E5000F0905D0540900E0950900F096090100968
:106E600070901109C301B2012EE036E040E050E01D
:106E70000E94644559016A016CE172E0E60EF71E5A
:106E80000027F7FC0095102FE21AF30A040B150BEC
:106E9000C801B70128E631E040E050E00E946445B7
:106EA000FB01E45BF04020919003309191032115A8
:106EB0003105F1F479E127163104D4F480916505A8
:106EC000909166058E0F9F1F9093660580936505D0
:106ED0008091B805882361F088EC90E09093D60407
:106EE0008093D504B0925F05A0925E051092B8051C
:106EF000C10168E070E00E942F456F5F7F4FCF01B6
:106F000043E0880F991F4A95E1F70E942F454B01F6
:106F1000AA2497FCA094BA2C840C951CA61CB71C20
:106F200080920E0990920F09A0921009B092110957
:106F30008091A203682E7724269CC001279C900D87
:106F4000369C900D112460E270E00E942F452301D1
:106F5000461A570A57FC79C02115310509F06EC051
:106F60008091990590919A05209197053091980507
:106F7000820F931F68E070E00E942F456B0180E450
:106F800090E0C80ED91E80915E0590915F05AA27FA
:106F900097FDA095BA2F0CE1E02E02E0F02E012D16
:106FA000112DE81AF90A0A0B1B0BC501B4012EE0DA
:106FB00036E040E050E00E946445E20EF31E041FFC
:106FC000151FC801B70128E631E040E050E00E94FB
:106FD0006445645B7040649DC001659D900D749D27
:106FE000900D1124B6010E942F459301220F331FEB
:106FF000260D371D2617370734F0309521953F4F62
:10700000621773070CF4B9019B01442737FD4095C3
:10701000542F8091500590915105A0915205B09147
:107020005305820F931FA41FB51F809350059093A3
:107030005105A0935205B09353050DC02150304027
:10704000309391032093900306C084EF91E09093D6
:107050009103809390038091B90581508093B90585
:107060008F3F09F09AC088E18093B905E0908F08BE
:10707000FF2400E010E06A817B818C819D81A80162
:1070800097010E9464453093EE072093ED076E81CF
:107090007F8188859985A80197010E946445309376
:1070A000F0072093EF0780910009909101099093D8
:1070B000F2078093F1078091120990911309909340
:1070C000F4078093F3078091040990910509909348
:1070D000F6078093F5078091790590917A05909352
:1070E000F8078093F70760915805709159058091D2
:1070F0005A0590915B0520E032E040E050E00E94AC
:1071000064453093FA072093F90780915C059091CC
:107110005D059093FE078093FD0780910E0390918B
:107120000F03909300088093FF0760910E09709100
:107130000F0980911009909111092EE036E040E08E
:1071400050E00E94644530932608209325088091E2
:107150006F0590E090932808809327088091460758
:1071600090E090931408809313088091D804909134
:10717000D90490931608809315088091E5059091A5
:10718000E60590932A08809329088091E70590915D
:10719000E80590932C0880932B089A859923A9F0F1
:1071A0006091DB087091DC08882777FD8095982F27
:1071B0000E94D5432091090930910A0940910B0999
:1071C00050910C090E948D442EC0E090DB08F09095
:1071D000DC086A817B818C819D810E94D54320914E
:1071E000F7083091F8084091F9085091FA080E9488
:1071F0008D445B016C010027F7FC0095102FC8013E
:10720000B7010E94D5432091090930910A094091A4
:107210000B0950910C090E948D449B01AC01C601E1
:10722000B5010E94D6420E94A2437093DC0860938D
:10723000DB08809182058823A9F06091D0087091C5
:10724000D108882777FD8095982F0E94D5432091FB
:10725000090930910A0940910B0950910C090E94CB
:107260008D442EC0E090D008F090D1086E817F81CF
:10727000888599850E94D5432091F7083091F808B8
:107280004091F9085091FA080E948D445B016C010D
:107290000027F7FC0095102FC801B7010E94D543C5
:1072A0002091090930910A0940910B0950910C096C
:1072B0000E948D449B01AC01C601B5010E94D642DB
:1072C0000E94A2437093D1086093D0086091040992
:1072D000709105092091F7083091F8084091F9085C
:1072E0005091FA082B873C874D875E87882777FD6A
:1072F0008095982F0E94D5437B018C0160910909EC
:1073000070910A0980910B0990910C099B01AC01C5
:107310000E94D6429B01AC01C801B7010E948D4476
:107320007B018C0160913C0570913D0580913E058B
:1073300090913F050E94D5432B853C854D855E8508
:107340000E948D4420E030E040E05FE30E948D44E5
:107350009B01AC01C801B7010E94D6420E94A24322
:1073600070930509609304098091DB089091DC0813
:1073700090931808809317088091D0089091D108B5
:1073800090931A08809319088091DB089091DC088B
:107390008150904434F080E090E49093DC08809336
:1073A000DB088091DB089091DC088050904C34F42D
:1073B00080E090EC9093DC088093DB088091D0080B
:1073C0009091D1088150904434F080E090E4909303
:1073D000D1088093D0088091D0089091D108805036
:1073E000904C34F480E090EC9093D1088093D008D6
:1073F00080910409909105098150904434F080E017
:1074000090E4909305098093040980910409909178
:1074100005098050904C34F480E090EC909305097D
:10742000809304098B889C88880C991C880C991C73
:107430008091830880FFC9C040919F0381FF0EC0E7
:10744000423310F58091790590917A054497909395
:107450007C0580937B051092630519C02091AA03D7
:107460003091AB03240F311D8091880890E0FC011E
:107470002E9FC0012F9F900D3E9F900D1124449789
:1074800090937C0580937B0581E080936305F9816F
:10749000FF2321F010927C0510927B052091790545
:1074A00030917A0540917B0550917C054217530736
:1074B0000CF08BC080916305882309F486C080910D
:1074C000A00390E0241B350BAC01429FC001439FF9
:1074D000900D529F900D112464E070E00E942F45A2
:1074E0005B01C090EF04D090F0046091580570915A
:1074F000590580915A0590915B05E090A103FF2406
:1075000000E010E020E830E040E050E00E946445F8
:10751000C801B7010E94F04420E230E040E050E0B2
:107520000E9464455EEF283E350714F428EE3EEFD6
:107530008091BA059091BB05FC01A4E0EE0FFF1FFE
:10754000AA95E1F7E81BF90BC60162E070E00E9422
:107550002F45E61BF70B61E02931360714F028E1CF
:1075600031E0E21BF30BC4018A199B098E0F9F1FA8
:1075700060E170E00E942F457093BB056093BA05EF
:107580008091840890E0880F991F880F991F6817D1
:10759000790764F4881699062CF09093BB058093C4
:1075A000BA0504C09092BB058092BA058091BA05D5
:1075B0009091BB058816990624F49092BB058092A1
:1075C000BA058090BA059090BB0580910309482EBA
:1075D00055248201000F111F000F111FC801805593
:1075E00090403401881599050CF43C017092FC0719
:1075F0006092FB078091040990910509298D3A8DCD
:107600004B8D5C8D62E0220F331F441F551F6A951E
:10761000D1F7821B930B31EA63167104ACF093012E
:1076200035952795821793070CF49C01C30162E0FE
:1076300070E00E942F45709561957F4FC901261714
:1076400037076CF4CB010BC04FEF803B940714F469
:1076500080EB9FEF8135910514F080E590E0980173
:1076600026193709281739070CF4C9019301201B83
:10767000310B4C01821793070CF449018091DB0810
:107680009091DC0820907005309071058219930963
:107690009093E9088093E80820E030E040E050E073
:1076A0006B857C858D859E850E9410448823C1F161
:1076B0006091D9057091DA058091DB059091DC0528
:1076C0000E94D5435B016C016A817B818C819D8125
:1076D0000E94D5432B853C854D855E850E948D4457
:1076E0007B018C01B101882777FD8095982F0E943E
:1076F000D5439B01AC01C801B7010E94D5429B0153
:10770000AC01C601B5010E94D6420E94A24360931B
:10771000D9057093DA058093DB059093DC051CC0D6
:107720002091E8083091E908442737FD4095542F0F
:107730008091D9059091DA05A091DB05B091DC0527
:10774000820F931FA41FB51F8093D9059093DA056C
:10775000A093DB05B093DC058091D9059091DA0503
:10776000A091DB05B091DC0581509A4FA040B0405C
:1077700064F080E09AEFA0E0B0E08093D9059093A8
:10778000DA05A093DB05B093DC058091D9059091D3
:10779000DA05A091DB05B091DC0580509640AF4F33
:1077A000BF4F64F480E096E0AFEFBFEF8093D90560
:1077B0009093DA05A093DB05B093DC056091E808AF
:1077C0007091E90880919A0390919B03A0919C038A
:1077D000B0919D038D8B9E8BAF8BB88F882777FDE3
:1077E0008095982F0E94D5437B018C016091D9052B
:1077F0007091DA058091DB059091DC050E94D543FC
:107800009B01AC016D897E898F89988D0E948D4482
:107810009B01AC01C801B7010E94D6420E94A2435D
:107820007B018C016B01C40197FE04C08827992756
:107830008819990962E070E00E942F45660D771D56
:10784000882777FD8095982F2091A90330E040E0AC
:1078500050E00E94F04420E430E040E050E00E941C
:107860006445388B2F87C216D3060CF497012F84FA
:1078700038883094219431083394221533050CF460
:107880009101C901880F991F880F991F67E070E067
:107890000E942F457A8B698B8091D0089091D108F6
:1078A000E0917205F0917305F8AFEFAB8E1B9F0B63
:1078B0009093CF088093CE0820E030E040E050E085
:1078C0006B857C858D859E850E9410448823D1F12F
:1078D0006091D5057091D6058091D7059091D80516
:1078E0000E94D5435B016C016E817F8188859985FB
:1078F0000E94D5432B853C854D855E850E948D4435
:107900007B018C012FA938ADB901882777FD8095BF
:10791000982F0E94D5439B01AC01C801B7010E947A
:10792000D5429B01AC01C601B5010E94D6420E941E
:10793000A2436093D5057093D6058093D7059093A5
:10794000D8051CC02091CE083091CF08442737FDC0
:107950004095542F8091D5059091D605A091D705DB
:10796000B091D805820F931FA41FB51F8093D50532
:107970009093D605A093D705B093D8058091D505EF
:107980009091D605A091D705B091D80581509A4F16
:10799000A040B04064F080E09AEFA0E0B0E08093B7
:1079A000D5059093D605A093D705B093D8058091BF
:1079B000D5059091D605A091D705B091D8058050F6
:1079C0009640AF4FBF4F64F480E096E0AFEFBFEF5B
:1079D0008093D5059093D605A093D705B093D8058D
:1079E0006091CE087091CF08882777FD8095982FF9
:1079F0000E94D5437B018C016091D5057091D6051D
:107A00008091D7059091D8050E94D5439B01AC0188
:107A10006D897E898F89988D0E948D449B01AC0170
:107A2000C801B7010E94D6420E94A2432F8538891F
:107A3000621773070CF49B01C901221533050CF47E
:107A4000C10163E070E00E942F458B0129893A89CA
:107A5000260D371DCB0162E070E00E942F455B01CF
:107A60007B01E818F908C701820F931F64E070E0FA
:107A70000E942F4577FF03C060E070E004C0461607
:107A800057060CF4B2018091DF08C82EDD246C1576
:107A90007D050CF4B6016093E7082A193B09C9017A
:107AA000880D991D64E070E00E942F4577FF03C0A8
:107AB00060E070E004C0461657060CF4B2016C1585
:107AC0007D050CF4B60160931609930169897A89E2
:107AD000261B370BC701820F931F64E070E00E94E2
:107AE0002F4577FF03C060E070E004C046165706DC
:107AF0000CF4B2016C157D050CF4B6016093D90845
:107B00002A193B09C901880D991D64E070E00E94A3
:107B10002F4577FF03C060E070E004C046165706AB
:107B20000CF4B2016C157D050CF4B6016093DD0810
:107B3000C301801B910B8819990964E070E00E94D1
:107B40002F4577FF03C060E070E004C0461657067B
:107B50000CF4B2016C157D050CF4B6016093FB08C2
:107B6000860C971CC401800F911F64E070E00E9496
:107B70002F4577FF03C060E070E004C0461657064B
:107B80000CF4B2016C157D050CF4B6016093FD0890
:107B9000E8960FB6F894DEBF0FBECDBFDF91CF9150
:107BA0001F910F91FF90EF90DF90CF90BF90AF901B
:107BB0009F908F907F906F905F904F903F902F900D
:107BC00008958091ED059091EE05A091EF05B0919B
:107BD000F0058093F5059093F605A093F705B09313
:107BE000F8058091F1059091F205A091F305B0910F
:107BF000F4058093F9059093FA05A093FB05B093E3
:107C0000FC0508951092E6051092E5051092E8052E
:107C10001092E705089584B1806A84B93D9A82E59F
:107C20008CBD1DBC459A81E0809319098AEA809336
:107C30001D0983E880931E098AE080931F09109232
:107C40002109109220091092230910922209109202
:107C50003F090895F8946091200570912105809165
:107C60002205909123052CE630E040E050E00E9490
:107C70006445309321092093200960912805709173
:107C8000290580912A0590912B052CE630E040E0F3
:107C900050E00E94644530932309209322096091AB
:107CA0000E0970910F0980911009909111092EE031
:107CB00036E040E050E00E9464453093290920936B
:107CC000280920911805309119058091EE089091AE
:107CD000EF08B9010E942F45CB01880F991F860F2D
:107CE000971F880F991F880F991F909325098093DC
:107CF00024098091070990910809B9010E942F4534
:107D0000CB01880F991F860F971F880F991F880F27
:107D1000991F9093270980932609109219051092B4
:107D200018051092EF081092EE08109208091092B0
:107D3000070980911F098B3009F468C08C3020F44A
:107D40008A3009F0DDC007C08C3009F4D0C08D3016
:107D500009F0D6C039C080918705809330098091A1
:107D6000880580933109809189058093320980913B
:107D70008A058093330980918B0580933409809123
:107D80008C058093350980918D058093360980910B
:107D90008E058093370980919D0580933809837FF4
:107DA00080939D0580910E0390910F038093390974
:107DB0008091930880933A09A2E0B0E00E94B64512
:107DC000802D80933B099CC08091DA088093300914
:107DD00080911409809331098091D20880933209EF
:107DE0008091DE08809333098091180980933409CB
:107DF0008091E008809335098091B9088093360915
:107E00008091BA08809337098FE06EC0E0917D08B9
:107E1000F0E0EE0FFF1FE35BF74F0190F081E02DE4
:107E20002FEFE138F20714F4E1E8FFEFE038F10555
:107E300014F0EFE7F0E0E0933009E0917E08F0E025
:107E4000EE0FFF1FE35BF74F0190F081E02D6FEF26
:107E5000E138F60714F4E1E8FFEFE038F10514F03B
:107E6000EFE7F0E0E0933109E0917C08F0E0EE0FFD
:107E7000FF1FE35BF74F0190F081E02D8FEFE138BA
:107E8000F80714F4E1E8FFEFE038F10514F0EFE74C
:107E9000F0E0E0933209E0917B08F0E0EE0FFF1F85
:107EA000E35BF74F0190F081E02D2FEFE138F2070F
:107EB00014F4E1E8FFEFE038F10514F0EFE7F0E04B
:107EC000E0933309809167058093340980916905B7
:107ED0008093350980916B058093360980916D05FB
:107EE0008093370980916F058093380909C080918C
:107EF0004607863018F01092460785E080933009D7
:107F0000789480913F09882309F456C04091410933
:107F100050914209CA0181509E4F8F5F9340B0F447
:107F20002091430930914409C90181509E4F8F5FD0
:107F3000934060F48091830885FF08C05093E60564
:107F40004093E5053093E8052093E70580914709C4
:107F50009091480921E08936920724F490935D05B9
:107F600080935C0580915C0590915D0520915E0594
:107F700030915F05845E9D4F821B930B68E671E034
:107F80000E942F45845B904090936105809360052B
:107F900080914B09282F30E08091D5049091D60430
:107FA0008217930788F480914607882369F43093F9
:107FB000D6042093D50408951092E6051092E505A5
:107FC0001092E8051092E705089580911909882319
:107FD00009F43BC045988DE199E090931B0980938B
:107FE0001A099091FD05E92FF0E0E455FC4F8081DE
:107FF00080931F099F5F9093FD05953010F01092BC
:10800000FD05109219090E942A3E81E080931C0907
:108010000000000000000000000000000000000060
:108020000000000000000000000000000000000050
:108030000000000000000000000000000000000040
:1080400080911D0980933C098EBD08958091190986
:10805000882309F07CC00DB407FE79C084E08093CA
:10806000D704459A2EB58091FF05813069F08130A3
:1080700018F08230C9F513C010923E092093FE0516
:10808000213891F581E008C0253541F58091FE0544
:108090008B5A8093FE0582E08093FF0525C0809176
:1080A0003E09E82FF0E0E75AF64F20838F5F809378
:1080B0003E099091FE058931A0F0291769F4A0E4EA
:1080C000B9E0E9E5F9E089E101900D928150E1F72D
:1080D00081E080933F0902C010923F091092FF0592
:1080E00003C0920F9093FE0520911C09203208F0E6
:1080F00028C04598000000000000000000000000BB
:10810000000000000000000000000000000000006F
:10811000000000000000000000000000000000005F
:1081200000000000E0911A09F0911B09E20FF11D17
:1081300080818EBD808190913C09890F80933C099C
:1081400003C081E0809319092F5F20931C090895D3
:1081500087B18C6087B9429843981092040680E8F2
:108160008093B103109205068093B2030895809125
:1081700006068150809306068F3F09F068C084E0B0
:10818000809306068091B0088B3F80F08091F008C4
:10819000873E28F08091AF0888231CF124C08A30E4
:1081A00028F48091AF088823F4F01BC08091040666
:1081B0008150809304068F3FB9F48091F00881507C
:1081C000809304068091B103813011F480E801C0EE
:1081D00086958093B1038091AF089091B103892374
:1081E00011F0429A01C042988091B2088B3F88F00A
:1081F00080910209873E28F08091B108882324F1FC
:1082000006C08A3030F48091B10887FF1DC04398C2
:108210000895809105068150809305068F3FB9F43B
:10822000809102098150809305068091B2038130CC
:1082300011F480E801C086958093B2038091B10863
:108240009091B203892311F0439A089543980895B9
:10825000A8E0B0E0EEE2F1E40C9489457B018C01EA
:10826000611571058105910519F482E089835AC071
:1082700083E089838EE1C82ED12CDC82CB82ED8213
:10828000FE820F831887C801B7010E949B41BC0181
:108290006150704077FF33C0EE27FF27E61BF70BD6
:1082A00020E030E040E050E081E090E0A0E0B0E08D
:1082B0000E2E04C0880F991FAA1FBB1F0A94D2F765
:1082C0000197A109B1098E219F21A023B123009715
:1082D000A105B10521F021E030E040E050E004C00C
:1082E00016950795F794E794EA95D2F72E293F293A
:1082F000402B512B2D833E834F8358870FC0611530
:10830000710581F0062E04C0EE0CFF1C001F111F2A
:108310000A94D2F7ED82FE820F831887C61AD70A15
:10832000DC82CB821A82CE0101960E94E841E8E00D
:1083300028960C94A545EF92FF920F931F939B01F3
:10834000AC01203080E0380781E0480780E0580722
:1083500080F42F3F31054105510509F020F4EE244A
:10836000FF24870119C068E0E62EF12C012D112DA4
:1083700013C0203080E0380780E0480781E05807CC
:1083800030F490E1E92EF12C012D112D05C088E18A
:10839000E82EF12C012D112D80E290E0A0E0B0E05C
:1083A0008E199F09A00BB10B04C0569547953795C0
:1083B0002795EA94D2F7F901ED54FC4F2081821BF6
:1083C0009109A109B1091F910F91FF90EF900895B4
:1083D0009F92AF92BF92CF92DF92EF92FF920F9354
:1083E0001F93EE24FF248701FC01248135814681FF
:1083F000578191808081823010F44061A2C0843026
:1084000009F49BC0823029F420E030E040E050E0E5
:1084100005C0211531054105510519F4E0E0F0E0F2
:1084200092C0828193816FEF823896070CF05AC018
:1084300062E87FEF681B790B6A3171052CF020E050
:1084400030E040E050E02AC0AA24BB24650181E06E
:1084500090E0A0E0B0E0062E04C0880F991FAA1F8C
:10846000BB1F0A94D2F70197A109B1098223932374
:10847000A423B5230097A105B10529F071E0A72E2B
:10848000B12CC12CD12C04C0569547953795279512
:108490006A95D2F72A293B294C295D29DA01C901BD
:1084A0008F779070A070B07080349105A105B105F0
:1084B00039F427FF09C0205C3F4F4F4F5F4F04C086
:1084C000215C3F4F4F4F5F4F80E090E0203060E0F5
:1084D000360760E0460760E4560710F081E090E060
:1084E000FC0123C08038910544F5FC01E158FF4FA1
:1084F000DA01C9018F779070A070B0708034910557
:10850000A105B10539F427FF09C0205C3F4F4F4F4B
:108510005F4F04C0215C3F4F4F4F5F4F57FF05C077
:108520005695479537952795319687E05695479507
:10853000379527958A95D1F706C020E030E040E0D6
:1085400050E0EFEFF0E0E22EF32E942F9F77802F94
:108550008078892B9E2F9795992797958F77082F4D
:10856000092B9E2F9695812F8078892B979499249B
:1085700097948F77182F1929C801B7011F910F9170
:10858000FF90EF90DF90CF90BF90AF909F900895B5
:10859000FC014150504030F001900616D1F7319760
:1085A000CF0108958827992708955058BB27AA27F7
:1085B0000ED079C16AD130F06FD120F031F49F3FF5
:1085C00011F41EF45FC10EF4E095E7FB55C1E92FED
:1085D0007BD180F3BA17620773078407950718F0F9
:1085E00071F49EF593C10EF4E0950B2EBA2FA02DD9
:1085F0000B01B90190010C01CA01A0011124FF2750
:10860000591B99F0593F50F4503E68F11A16F0404A
:10861000A22F232F342F4427585FF3CF4695379549
:108620002795A795F0405395C9F77EF41F16BA0B0E
:10863000620B730B840BBAF09150A1F0FF0FBB1FBC
:10864000661F771F881FC2F70EC0BA0F621F731F05
:10865000841F48F4879577956795B795F7959E3F62
:1086600008F0B3CF9395880F08F09927EE0F9795F0
:10867000879508950CD017C10FD140F006D130F086
:1086800021F45F3F19F0F8C0511141C1FBC01CD16A
:1086900098F39923C9F35523B1F3951B550BBB27C9
:1086A000AA2762177307840738F09F5F5F4F220F76
:1086B000331F441FAA1FA9F333D00E2E3AF0E0E86F
:1086C00030D091505040E695001CCAF729D0FE2FBB
:1086D00027D0660F771F881FBB1F2617370748074D
:1086E000AB07B0E809F0BB0B802DBF01FF27935803
:1086F0005F4F2AF09E3F510568F0BEC008C15F3F42
:10870000ECF3983EDCF3869577956795B795F795EA
:108710009F5FC9F7880F911D9695879597F90895E2
:10872000E1E0660F771F881FBB1F6217730784077E
:10873000BA0720F0621B730B840BBA0BEE1F88F78D
:10874000E095089504D06894B111E1C00895C4D0B3
:1087500088F09F5790F0B92F9927B751A0F0D1F02A
:10876000660F771F881F991F1AF0BA95C9F712C0B4
:10877000B13081F0CBD0B1E00895C8C0672F782F19
:108780008827B85F39F0B93FCCF386957795679520
:10879000B395D9F73EF490958095709561957F4F8C
:1087A0008F4F9F4F0895E89409C097FB3EF4909532
:1087B0008095709561957F4F8F4F9F4F9923A9F0BA
:1087C000F92F96E9BB279395F69587957795679549
:1087D000B795F111F8CFFAF4BB0F11F460FF1BC08D
:1087E0006F5F7F4F8F4F9F4F16C0882311F096E920
:1087F00011C0772321F09EE8872F762F05C06623CE
:1088000071F096E8862F70E060E02AF09A95660F86
:10881000771F881FDAF7880F9695879597F908953F
:1088200007D008F481E0089503D008F48FEF08958D
:10883000990F0008550FAA0BE0E8FEEF1616170671
:10884000E807F907C0F012161306E407F50798F0D9
:10885000621B730B840B950B39F40A2661F0232BF2
:10886000242B252B21F408950A2609F4A140A6956E
:108870008FEF811D811D089597F99F6780E870E053
:1088800060E008959FEF80EC089500240A94161686
:10889000170618060906089500240A9412161306EE
:1088A000140605060895092E0394000C11F488237C
:1088B00052F0BB0F40F4BF2B11F460FF04C06F5F98
:1088C0007F4F8F4F9F4F089557FD9058440F551F6E
:1088D00059F05F3F71F04795880F97FB991F61F042
:1088E0009F3F79F087950895121613061406551FB9
:1088F000F2CF4695F1DF08C0161617061806991F25
:10890000F1CF86957105610508940895E894BB2719
:1089100066277727CB0197F908950BD0C4CFB5DF31
:1089200028F0BADF18F0952309F0A6CFABCF1124B9
:10893000EECFCADFA0F3959FD1F3950F50E0551FFE
:10894000629FF001729FBB27F00DB11D639FAA27A4
:10895000F00DB11DAA1F649F6627B00DA11D661FF3
:10896000829F2227B00DA11D621F739FB00DA11D14
:10897000621F839FA00D611D221F749F3327A00DCE
:10898000611D231F849F600D211D822F762F6A2F6A
:1089900011249F5750408AF0E1F088234AF0EE0FEF
:1089A000FF1FBB1F661F771F881F91505040A9F7FC
:1089B0009E3F510570F060CFAACF5F3FECF3983E29
:1089C000DCF3869577956795B795F795E7959F5F63
:1089D000C1F7FE2B880F911D9695879597F90895FD
:1089E000629FD001739FF001829FE00DF11D649F93
:1089F000E00DF11D929FF00D839FF00D749FF00D1F
:108A0000659FF00D9927729FB00DE11DF91F639FBF
:108A1000B00DE11DF91FBD01CF0111240895991B6F
:108A200079E004C0991F961708F0961B881F7A9565
:108A3000C9F780950895AA1BBB1B51E107C0AA1F67
:108A4000BB1FA617B70710F0A61BB70B881F991FEF
:108A50005A95A9F780959095BC01CD01089597FB93
:108A6000092E07260AD077FD04D0E5DF06D00020C6
:108A70001AF4709561957F4F0895F6F7909581955A
:108A80009F4F0895A1E21A2EAA1BBB1BFD010DC02A
:108A9000AA1FBB1FEE1FFF1FA217B307E407F507AE
:108AA00020F0A21BB30BE40BF50B661F771F881F8A
:108AB000991F1A9469F760957095809590959B0120
:108AC000AC01BD01CF01089597FB092E05260ED0FC
:108AD00057FD04D0D7DF0AD0001C38F450954095DC
:108AE000309521953F4F4F4F5F4F0895F6F7909582
:108AF0008095709561957F4F8F4F9F4F08952F926E
:108B00003F924F925F926F927F928F929F92AF921D
:108B1000BF92CF92DF92EF92FF920F931F93CF936A
:108B2000DF93CDB7DEB7CA1BDB0B0FB6F894DEBF01
:108B30000FBECDBF09942A88398848885F846E8427
:108B40007D848C849B84AA84B984C884DF80EE8071
:108B5000FD800C811B81AA81B981CE0FD11D0FB67A
:108B6000F894DEBF0FBECDBFED010895F999FECF99
:108B7000B2BDA1BDF89A119600B40895F999FECF3F
:108B8000B2BDA1BD00BC11960FB6F894FA9AF99A3D
:068B90000FBE0895FFCFA7
:108B96000A010101FF64496E74656772616C4E6972
:108BA600636B20202020496E74656772616C526F7A
:108BB6006C6C202020204163634E69636B2020206B
:108BC600202020202020416363526F6C6C202020DF
:108BD6002020202020204779726F47696572202067
:108BE600202020202020486F6568656E57657274C6
:108BF6002020202020204163635A2020202020208E
:108C060020202020202047617320202020202020A3
:108C16002020202020204B6F6D7061737356616C8D
:108C26007565202020205370616E6E756E6720205A
:108C36002020202020204D6F746F7220564C20205B
:108C46002020202020204D6F746F72205652202045
:108C56002020202020204D6F746F7220484C202049
:108C66002020202020204D6F746F72204852202033
:108C76002020202020204D6F746F72204C696E6B6F
:108C86007320202020204D6F746F72205265636818
:108C96007473202020202020202020202020202027
:108CA60020202020202044697374616E6365202093
:108CB6002020202020204F73644261722020202033
:108CC6002020202020204D4B334D61672043616CCE
:108CD600537461746520536572766F2020202020BE
:108CE6002020202020204E69636B20202020202079
:108CF600202020202020526F6C6C20202020202055
:108D0600202020202020202020202020202020205D
:108D1600202020202020202020202020202020204D
:108D2600202020202020202020202020202020203D
:108D3600202020202020202020202020202020202D
:108D4600202020202020202020202020202020201D
:108D560020202020202045727361747A6B6F6D701D
:108D6600617373202020456D7066616E6720202038
:108D76002020202020204750535F4E69636B20201F
:108D86002020202020204750535F526F6C6C2020FB
:108D96002020202020202800FFFF6400800164009E
:108DA600007D0000FF0373737301020304050607C9
:108DB60008090A48616C6C6F2057656C74000000E6
:108DC600000000000000000000000000000000009D
:108DD600000000000000000000000000000000008D
:108DE600000000000000000000000000000000007D
:108DF600000000000000000000000000000000006D
:108E06000000000B01426567696E6E657200004ED8
:108E16006F726D616C000053706F727400006400B5
:108E2600F40190D0030090D0030017B7D13830FB7F
:108E3600103A409696020A644664ECFF0A0B0D0B44
:108E46000C010100010202030303030404040404E9
:108E560004040405050505050505050505050505BF
:108E6600050505060606060606060606060606069F
:108E7600060606060606060606060606060606068C
:108E8600060606070707070707070707070707076F
:108E9600070707070707070707070707070707075C
:108EA600070707070707070707070707070707074C
:108EB600070707070707070707070707070707073C
:108EC600070707080808080808080808080808081F
:108ED600080808080808080808080808080808080C
:108EE60008080808080808080808080808080808FC
:108EF60008080808080808080808080808080808EC
:108F060008080808080808080808080808080808DB
:108F160008080808080808080808080808080808CB
:108F260008080808080808080808080808080808BB
:108F360008080808080808080808080808080808AB
:048F4600080808000F
:00000001FF
